:100000000263340258F0AB07AA06900000C3E582F1
:100010009BEA6480F8E58364809850061276B9A361
:1000200080EB22026F927F15026A8C026773900E3A
:10003000677401F0A3740DF0A37433F0900E66742E
:100040000AF022025799E709F608DFFA8046E70925
:10005000F208DFFA803E88828C83E709F0A3DFFA9A
:100060008032E309F608DFFA8078E309F208DFFA64
:10007000807088828C83E309F0A3DFFA8064898230
:100080008A83E0A3F608DFFA805889828A83E0A396
:10009000F208DFFA804C80D280FA80C680D4806972
:1000A00080F28033801080A680EA809A80A880DA6F
:1000B00080E280CA803389828A83ECFAE493A3C801
:1000C000C582C8CCC583CCF0A3C8C582C8CCC583C3
:1000D000CCDFE9DEE7800D89828A83E493A3F6080A
:1000E000DFF9ECFAA9F0EDFB2289828A83ECFAE0D1
:1000F000A3C8C582C8CCC583CCF0A3C8C582C8CC70
:10010000C583CCDFEADEE880DB89828A83E493A3BF
:10011000F208DFF980CC88F0EF60010E4E60C388F2
:10012000F0ED2402B4040050B9F582EB2402B404CB
:100130000050AF232345822390009673C2D530F739
:1001400007B2D563F0FF05F030E70CB2D5F40484B4
:1001500063F0FF05F080018430D502F40422BB0176
:100160000689828A83E0225002E722BBFE02E32254
:1001700089828A83E49322BB010989828A83F8E019
:1001800028F022500327F722BBFE05F8E328F322CC
:100190008A838982F8E4932822BB010689828A83B4
:1001A000F0225002F722BBFE01F322EF8DF0A4A84B
:1001B000F0CF8CF0A428CE8DF0A42EFE22C2D5EC78
:1001C00030E709B2D5E4C39DFDE49CFCEE30E715B1
:1001D000B2D5E4C39FFFE49EFE1205F8C3E49DFD83
:1001E000E49CFC80031205F830D507C3E49FFFE4CC
:1001F0009EFE22C5F0F8A3E028F0C5F0F8E58215D0
:100200008270021583E038F022A3F8E0C5F025F0F3
:10021000F0E582158270021583E0C838F0E822BB51
:10022000010A89828A83E0F5F0A3E022500687F074
:1002300009E71922BBFE07E3F5F009E319228982D9
:100240008A83E493F5F074019322BB010A89828AC0
:1002500083F0E5F0A3F0225006F709A7F01922BBBE
:10026000FE06F3E5F009F31922E88FF0A4CC8BF039
:10027000A42CFCE98EF0A42CFC8AF0EDA42CFCEA62
:100280008EF0A4CDA8F08BF0A42DCC3825F0FDE99C
:100290008FF0A42CCD35F0FCEB8EF0A4FEA9F0EB92
:1002A0008FF0A4CFC5F02ECD39FEE43CFCEAA42D9E
:1002B000CE35F0FDE43CFC2275F008758200EF2F8E
:1002C000FFEE33FECD33CDCC33CCC58233C5829B1C
:1002D000ED9AEC99E58298400CF582EE9BFEED9A42
:1002E000FDEC99FC0FD5F0D6E4CEFBE4CDFAE4CCDE
:1002F000F9A88222B800C1B90059BA002DEC8BF0E0
:1003000084CFCECDFCE5F0CBF97818EF2FFFEE339C
:10031000FEED33FDEC33FCEB33FB10D703994004C7
:10032000EB99FB0FD8E5E4F9FA227818EF2FFFEEEE
:1003300033FEED33FDEC33FCC933C910D7059BE91F
:100340009A4007EC9BFCE99AF90FD8E0E4C9FAE47B
:10035000CCFB2275F010EF2FFFEE33FEED33FDCC1A
:1003600033CCC833C810D7079BEC9AE899400AED04
:100370009BFDEC9AFCE899F80FD5F0DAE4CDFBE4AC
:10038000CCFAE4C8F922EB9FF5F0EA9E42F0E99D31
:1003900042F0E89C45F022E8600FECC313FCED133B
:1003A000FDEE13FEEF13FFD8F122E8600FEFC33329
:1003B000FFEE33FEED33FDEC33FCD8F122ECF0A37D
:1003C000EDF0A3EEF0A3EFF022D083D082F8E49317
:1003D0007012740193700DA3A393F8740193F582C6
:1003E0008883E4737402936860EFA3A3A380DF8A19
:1003F000838982E473EC8EF0A4CCC5F0CCCDF8EF09
:10040000A4CEC5F02DFDE43CFCE8A42EC8C5F03D0B
:10041000FDE43CFCEFA4FFE5F028FEE43DFDE43CF8
:10042000FC22E3F5F009E208B5F06BDFF58067E345
:10043000F5F009E608B5F05EDFF5805A87F009E6C9
:1004400008B5F052DFF6804E87F009E208B5F046B5
:10045000DFF6804288828C8387F009E0A3B5F0360E
:10046000DFF6803288828C8387F009E493A3B5F0AD
:1004700025DFF5802188828C83E3F5F009E0A3B5C0
:10048000F014DFF5801088828C83E3F5F009E493A3
:10049000A3B5F002DFF4020551808780E9809080E7
:1004A000D4803E8015806E807E809D80B7808D8058
:1004B000A380518074803C02055D89828A83ECFAB6
:1004C000E493F5F0A3C8C582C8CCC583CCE493A35C
:1004D000C8C582C8CCC583CCB5F076DFE3DEE18049
:1004E0007089828A83E493F5F0A3E208B5F062DFB5
:1004F000F4805E89828A83E0F5F0A3E608B5F051C6
:10050000DFF5804D89828A83E0F5F0A3E208B5F03B
:1005100040DFF5803C89828A83E493F5F0A3E60806
:10052000B5F02EDFF4802A8002805789828A83EC1E
:10053000FAE493F5F0A3C8C582C8CCC583CCE0A388
:10054000C8C582C8CCC583CCB5F006DFE4DEE28046
:10055000007FFFB5F0020F2240027F012289828ACC
:1005600083ECFAE0F5F0A3C8C582C8CCC583CCE023
:10057000A3C8C582C8CCC583CCB5F0D5DFE5DEE322
:1005800080CF89828A83ECFAE0F5F0A3C8C582C8DF
:10059000CCC583CCE493A3C8C582C8CCC583CCB5F5
:1005A000F0AFDFE4DEE280A988F0EF60010E4E607C
:1005B000ABED2402B404005098F582EB2402B4049D
:1005C00000508E232345822390049973EF4E6012CE
:1005D000EF60010EEDBB010B89828A83F0A3DFFC83
:1005E000DEFA2289F05007F709DFFCA9F022BBFEF2
:1005F000FCF309DFFCA9F022BC000BBE0029EF8D43
:10060000F084FFADF022E4CCF875F008EF2FFFEE98
:1006100033FEEC33FCEE9DEC984005FCEE9DFE0FA6
:10062000D5F0E9E4CEFD22EDF8F5F0EE8420D21C01
:10063000FEADF075F008EF2FFFED33FD4007985049
:1006400006D5F0F222C398FD0FD5F0EA22E4FFFEB2
:10065000FDFC900C5E1203BD900C5EE0F8A3E0F987
:10066000A3E0FAA3E0FB900E29E0FFE4FCFDFEEB23
:100670002FFFEE3AFEED39FDEC38FC900C5E1203D4
:10068000BD900C5EE0F8A3E0F9A3E0FAA3E0FBC0A4
:1006900000900E2AE0FFE4FCFDFE78081203AAD0C9
:1006A00000EB2FFFEA3EFEE93DFDE83CFC900C5ECE
:1006B0001203BD900C5EE0F8A3E0F9A3E0FAA3E01A
:1006C000FBC000900E2BE0FFE4FCFDFE781012034F
:1006D000AAD000EB2FFFEA3EFEE93DFDE83CFC908E
:1006E0000C5E1203BD900E28E024FE700302079AF0
:1006F00024FE70030207C524FC700302089424F84A
:1007000070030208EE14700302096E24F1700302F4
:100710000A53241F6003020B80900C5EE0FCA3E0F0
:10072000FDA3E0FEA3E0FF900C6B1203BD7F161249
:1007300017DF900C5D748BF01277C3900C5DE02492
:100740001BF0E0FF12470B900C62EFF0900C6F74FF
:1007500001F0A3740CF0A3745CF07B017A0C795B5C
:10076000E4FFFE123441900C5BE0540FC3940E4042
:100770000A900C5DE06480946C40C0127779900C14
:100780005BE0FE540F900D77F0EEC4540FA3F09091
:100790000C5CE0900D79F0020B88900C5EE0FCA3FD
:1007A000E0FDA3E0FEA3E0FF900C6B1203BD7F16FB
:1007B0001217DF122BA6AD07AC06EF900D77F0EE07
:1007C000A3F0020B88900007E004F0900B4CE004CB
:1007D000F0900007E0FBD39435400A7435F0E490C4
:1007E0000D77020B85900C5EE0FCA3E0FDA3E0FE1C
:1007F000A3E0FF75F004EBA42404F582E5F03400D7
:10080000F5831203BD900E2CE0FF74DB2BF582E420
:100810003400F583EFF0900E2DE0900B4DF0900C2E
:100820005EE0FCA3E0FDA3E0FEA3E0FF900003E098
:10083000F8A3E0F9A3E0FAA3E0FBC3120386501487
:10084000900C5EE0FCA3E0FDA3E0FEA3E0FF9000BF
:10085000031203BD900C5EE0FCA3E0FDA3E0FEA349
:10086000E0FF900B48E0F8A3E0F9A3E0FAA3E0FB77
:10087000D31203864014900C5EE0FCA3E0FDA3E0DD
:10088000FEA3E0FF900B481203BD900D7774FCF0BF
:10089000A30209689000077401F0900B4CF0900CD3
:1008A0005EE0FCA3E0FDA3E0FEA3E0FF90000812E1
:1008B00003BD900E2CE09000DCF0900C5EE0FCA3F9
:1008C000E0FDA3E0FEA3E0FF9000031203BD900C47
:1008D0005EE0FCA3E0FDA3E0FEA3E0FF900B481266
:1008E00003BD900D7774FEF0A304F0020B88900E08
:1008F00029E0FF7E00900B41EEF0A3EFF0FD900E9B
:100900002AE0FFED900B41CFF0A3EFF0900E2BE02B
:10091000FF900B13EEF0A3EFF0FD900E2CE0FFED37
:10092000900B13CFF0A3EFF0900E2DE0FF900B355E
:10093000EEF0A3EFF0FD900E2EE0FFED900B35CF23
:10094000F0A3EFF0900D7774FEF0C3900B14E094D9
:1009500032900B13E09400500CE4F0A37432F0904A
:100960000D7774FFF0900D7874FFF0020B88E4FFB0
:10097000FEFDFC900C621203BD74FFFFFEFDFC90B7
:100980000C661203BD900D7774FEF0A304F0900B7B
:100990004DE0900D79F0900B41E0FCA3E0900D7AD2
:1009A000F0ECA3F0900B13E0FCA3E0900D7CF0ECD6
:1009B000A3F0900B35E0FCA3E0900D7EF0ECA3F0EB
:1009C000900B48E0FCA3E0FDA3E0FEA3E0FF900D48
:1009D00080EFF0900B48A3A3A3E078081203979050
:1009E0000D81EFF0900B48E0FCA3E0FDA3E0FEA337
:1009F000E0FF7810120397900D82EFF0900003E073
:100A0000FCA3E0FDA3E0FEA3E0FF900D83EFF090D8
:100A10000003A3A3A3E07808120397900D84EFF0DE
:100A2000900003E0FCA3E0FDA3E0FEA3E0FF78104C
:100A3000120397900D85EFF0900B4CE0900D86F02F
:100A40009000DCE0900D87F0900007E0900D88F0BA
:100A5000020B88900E2DE0FE900E2CE0FDEDFF9035
:100A60000C62EEF0A3EFF07F07127340900C64EF7E
:100A7000F07F08127340900C65EFF0E4FD7F0712E1
:100A800074C6E4FD7F081274C6900C5EE0FCA3E01F
:100A9000FDA3E0FEA3E0FF900C6B1203BD7F1612D6
:100AA00017DF900D757442F0A37440F0900E7CE057
:100AB000FBA3E0FAA3E02401F9E43AFA12015E9004
:100AC0000E7BF0A37401F0A3740DF0A37475F09085
:100AD0000D7774FEF0A304F07F42124DEA900C6291
:100AE000E0FEA3E0FFD394E8EE9403401BEF242044
:100AF000FFE43EFEEF7806CEC313CE13D8F9FF7C99
:100B0000007D301201AB801A900C62E0FEA3E0FF82
:100B10007C007D301201ABEF7806CEC313CE13D824
:100B2000F9FF900B39EEF0A3EFF0E4A3F01275D8C3
:100B30001278BA7F011273D97F8F1275FC7F9E12D3
:100B400075FC7D0A7C007F807E0012666CE4900B51
:100B500052F0A3F012753FEF60061278B4EF60D840
:100B6000E4FF1273D9900C64E0FD7F071274C69005
:100B70000C65E0FD7F081274C6900B407401F022F2
:100B8000900D7774FFF0A3F0900D757442F0A3748C
:100B900040F0900E7CE0FBA3E0FAA3E02401F9E42E
:100BA0003AFA12015E900E7BF0A37401F0A3740D6B
:100BB000F0A37475F07F42124DEA22E4900C55F0D8
:100BC000900C58F0A374C8F0A37401F053D9BF126D
:100BD0007839D2AF12724F1277D47BFF7A6479845E
:100BE0001210837F5E7EC67D0D7C0090000812038C
:100BF000BD9000DC74D8F07F527EC87D0D7C0090E3
:100C0000000C1203BD9000DD74D8F07F467ECA7DD3
:100C10000D7C009000101203BD9000DE74D8F07FB0
:100C20003A7ECC7D0D7C009000141203BD9000DF55
:100C300074D8F07F2E7ECE7D0D7C009000181203BC
:100C4000BD9000E074D8F07F227ED07D0D7C0090B6
:100C5000001C1203BD9000E174D8F07F167ED27D97
:100C60000D7C009000201203BD9000E274D8F07F4C
:100C70000A7ED47D0D7C009000241203BD9000E319
:100C800074D8F07FFE7ED57D0D7C00900028120385
:100C9000BD9000E474D8F07FF27ED77D0D7C00908B
:100CA000002C1203BD9000E574D8F07FE67ED97D5C
:100CB0000D7C009000301203BD9000E674D8F07FE8
:100CC000DA7EDB7D0D7C009000341203BD9000E7DE
:100CD00074D8F07FCE7EDD7D0D7C0090003812034D
:100CE000BD9000E874D8F07FC27EDF7D0D7C00905F
:100CF000003C1203BD9000E974D8F07FB67EE17D20
:100D00000D7C009000401203BD9000EA74D8F07F83
:100D1000AA7EE37D0D7C009000441203BD9000EBA1
:100D200074D8F07F9E7EE57D0D7C00900048120314
:100D3000BD9000EC74D8F07F927EE77D0D7C009032
:100D4000004C1203BD9000ED74D8F07F867EE97DE3
:100D50000D7C009000501203BD9000EE74D8F07F1F
:100D60007A7EEB7D0D7C009000541203BD9000EF65
:100D700074D8F07F6E7EED7D0D7C009000581203DC
:100D8000BD9000F074D8F07F627EEF7D0D7C009006
:100D9000005C1203BD9000F174D8F07F567EF17DA7
:100DA0000D7C009000601203BD9000F274D8F07FBB
:100DB0004A7EF37D0D7C009000641203BD9000F329
:100DC00074D8F07F3E7EF57D0D7C009000681203A4
:100DD000BD9000F474D8F07F327EF77D0D7C0090DA
:100DE000006C1203BD9000F574D8F07F267EF97D6B
:100DF0000D7C009000701203BD9000F674D8F07F57
:100E00001A7EFB7D0D7C009000741203BD9000F7EC
:100E100074D8F07F0E7EFD7D0D7C0090007812036B
:100E2000BD9000F874D8F07F027EFF7D0D7C0090AD
:100E3000007C1203BD9000F974D8F07F5C7E797D50
:100E40000C7C009000801203BD9000FA74D8F07FF3
:100E5000EA7E027D0E7C009000841203BD9000FBB0
:100E600074D8F07FDE7E047D0E7C00900088120333
:100E7000BD9000FC74D8F07FD27E067D0E7C009081
:100E8000008C1203BD9000FD74D8F07FC67E087DF3
:100E90000E7C009000901203BD9000FE74D8F07F8D
:100EA000BA7E0A7D0E7C009000941203BD9000FF74
:100EB00074D8F07FAE7E0C7D0E7C009000981203FB
:100EC000BD90010074D8F07FA27E0E7D0E7C009054
:100ED000009C1203BD90010174D8F07F967E107DB6
:100EE0000E7C009000A01203BD90010274D8F07F28
:100EF0008A7E127D0E7C009000A41203BD90010337
:100F000074D8F07F7E7E147D0E7C009000A81203C2
:100F1000BD90010474D8F07F727E167D0E7C009027
:100F200000AC1203BD90010574D8F07F667E187D79
:100F30000E7C009000B01203BD90010674D8F07FC3
:100F40005A7E1A7D0E7C009000B41203BD900107FA
:100F500074D8F07F4E7E1C7D0E7C009000B812038A
:100F6000BD90010874D8F07F427E1E7D0E7C0090FB
:100F700000BC1203BD90010974D8F07F367E207D3D
:100F80000E7C009000C01203BD90010A74D8F07F5F
:100F90002A7E227D0E7C009000C41203BD90010BBE
:100FA00074D8F07F1E7E247D0E7C009000C8120352
:100FB000BD90010C74D8F07F127E267D0E7C0090CF
:100FC00000CC1203BD90010D74D8F090000774326C
:100FD000F0A3E0FCA3E0FDA3E0FEA3E0FF121DB13F
:100FE000900C56EEF0A3EFF04E60177FE87E0312F0
:100FF0007641900C56A3E0FF125E947FE87E0312C8
:1010000076417BFF7A6479A0900C56E0FFA3E090D4
:101010000CDCCFF0A3EFF0121083127843126FDDD7
:101020007BFF7A6479C4121083900C58E07002A39D
:10103000E06010900C59E024FFF0900C58E034FF71
:10104000F0803B900C56E07002A3E07F0060027FCE
:101050000474C07E5DA807088005C333CE33CED8A4
:10106000F9900C59F0EE900C58F0900C5AE0600694
:10107000E4F0C2A28008900C5A7401F0D2A212735C
:10108000A680A6900CD9EBF0A3EAF0A3E9F0E490D7
:101090000D04F0A3F0A3F0A3F0A3F0A3F0A3F0A33A
:1010A000F0900D10F0A3F0A3F0A3F0A3F0900D1CAE
:1010B00004F0A3740CF0A374DCF0900CD9E0FBA353
:1010C000E0FAA3E0F912015E70030214BC1203C936
:1010D00014760A11132514123014383114383214CE
:1010E0003833143834143835143836143837143843
:1010F00038143839116A44116A55116258116A63FB
:10110000116A64113568116A6C116A75116A780088
:1011100000148CE4900D1AF0A3F0900D08E0700418
:10112000A3E06401900D087008F0A3F07F2502147D
:101130009BE4021421900D08E07002A3E06011907E
:101140000D1BE004F07006900D1AE004F002149EEE
:10115000900CD9E0FBA3E0FAA3E0F912015EFF02D4
:10116000149B900D12E4F0A304F0E4900D0CF0A396
:10117000F0A3F0A3F0900D08E07004A3E064016018
:10118000030213F6900D1FF0A37404F0900D1AE003
:10119000FEA3E0FF64024E7026900D1FF0A37402C0
:1011A000F0900D1CE0FBA3E475F001120209A9F018
:1011B000FA12015EFD900D06E4F0A3EDF08021EF40
:1011C00064014E900D1CE0FBA3E475F002120209CD
:1011D000A9F0FA12021FFF900D06E5F0F0A3EFF060
:1011E000900D1FE0FFA3E0900D04CFF0A3EFF0D32C
:1011F000900D05E09400900D04E09400500302135C
:1012000014900D1FA3E01425E025E0FD740F7E006F
:10121000A805088005C333CE33CED8F9FF900D065C
:10122000E05EFEA3E05FA805088005CEC313CE13E1
:10123000D8F9FF900D04E0FCA3E0FD2414F58274BE
:101240000D3CF583EFF074142DF582740D3CF5839D
:10125000E0FFC3940A402BEFD3940F5025900D125A
:10126000E07002A3E07E5760027E37EE2FFF900D04
:1012700004E0FCA3E02414F582740D3CF583EFF048
:101280008021900D04E0FEA3E0FF2414F582740D8C
:101290003EF583E02430FD74142FF582740D3EF585
:1012A00083EDF0900D04E0FEA3E02414F582740DAC
:1012B0003EF583E0B4302A900D0CE07002A3E0709C
:1012C00010900D0FE004F07026900D0EE004F080F9
:1012D0001E900D0DE004F07006900D0CE004F080FF
:1012E0000E900D0DE004F07006900D0CE004F090EF
:1012F0000D07E0C4F8540FC868F0900D06E0C45420
:10130000F048F0900D05E024FFF0900D04E034FF6C
:10131000F00211EF900D1FE0FEA3E0FF2415F5820F
:10132000740D3EF583E4F0900D08F0A3F0900D10DD
:10133000E07002A3E07008900D10EEF0A3EFF090C3
:101340000D0CE0FEA3E0FFC3900D11E09F900D1087
:10135000E09E4070E4900D04F0A3F0900D0CE0FED0
:10136000A3E0FFC3900D11E09FFF900D10E09EFEE3
:10137000C3900D05E09F900D04E09E50157F301244
:101380006F05900D05E004F070D1900D04E004F0BD
:1013900080C9900D0CE0FFA3E0900D04CFF0A3EF07
:1013A000F0900D04E0FEA3E0FFD39400EE94004023
:1013B00057126EF9900D05E024FFF0900D04E03413
:1013C000FFF080DD900D0CE0FFA3E0900D04CFF066
:1013D000A3EFF0900D04E0FEA3E0FFD39400EE94A1
:1013E000004025126EF9900D05E024FFF0900D04E9
:1013F000E034FFF080DD900CD9E0FBA3E0FAA3E03D
:10140000F912015EFF126F05E4900D10F0A3F0A336
:101410008051900D08E07004A3E064017009900D04
:101420000AF0A304F08077900CD9E0FBA3E0FAA3C4
:10143000E0F912015EFF8063900D0AE07004A3E002
:101440006401900CD97021E0FBA3E0FAA3E0F9124B
:10145000015E24D0FEE434FF900D10F0A3CEF0E442
:10146000900D0AF0A3F08036E0FBA3E0FAA3E0F9C8
:1014700012015EFF80257F0D126F05900CD9E0FBF5
:10148000A3E0FAA3E0F912015EFF800F900CD9E00F
:10149000FBA3E0FAA3E0F912015EFF126F05900CC6
:1014A000D9E0FBA3E0FAA3E02401F9E43AFA900CB6
:1014B000D9EBF0A3EAF0A3E9F00210BA22E59620F6
:1014C000E7FB75960EE4F597E59620E7FB75969198
:1014D000E59620E7FB900CD8E597F0900F2AE0B452
:1014E0000513E59620E7FBE4F596900F21E0F597CC
:1014F000E4900F2AF0900CD8E0FF30E210E596203F
:10150000E7FB759611E4F597900F2AF022EF30E48F
:101510001BE59620E7FB759611759708E59620E781
:10152000FB759611759780E4900F2AF0900F2AE0D2
:101530006003021629900CD8E020E0030216297BF4
:10154000017A0F791E7D087C007F20126C8C900F31
:1015500021E0FE900F20E07C002400FFEC3EF0A391
:10156000EFF0900F23E0FE900F22E02400FFEC3E0E
:10157000F0A3EFF0900F25E0FE900F24E02400FF91
:10158000EC3EF0A3EFF0900F1EE0547F6421703525
:10159000A3E024FE601B14602224FA600F1460167E
:1015A00014601D240A707F127028807D1270738071
:1015B0007812791A8073127765806E12791B8069B0
:1015C00012791C8064900F1FE0B40C0050589015E5
:1015D000D5F82828730215F90215FE021626021600
:1015E0000302162602160802160D0216260216120D
:1015F00002161702161C02162112529E802B12652B
:101600006280261263C38021126EA8801C1238ECFF
:1016100080171266F180121264D8800D126A24803D
:101620000812728B800312769C900F2AE06401608E
:10163000030216FC900CD8E030E1030216FCE5969C
:1016400020E7FB759691E59620E7FB900CD8E5978F
:10165000F0E030E40630E0030216FC900CD874028F
:10166000F0C3900F29E09440900F28E09400403C94
:10167000900F1BE0FBA3E0FAA3E0F97D407C007F24
:1016800020126E51900F1CE475F0401201F3900F80
:1016900029E024C0F0900F28E034FFF0900F27E0FD
:1016A0002440F0900F26E03400F08024900F28E0D2
:1016B000FCA3E0FD900F1BE0FBA3E0FAA3E0F97FA1
:1016C00020126E51900CD8E04408F0E4900F2AF0FC
:1016D000900F24E0FEA3E0FFA3E0B50611A3E0B560
:1016E000070C900CD8E04408F0E4900F2AF0E5963F
:1016F00020E7FB759611900CD8E0F597900F2AE043
:10170000640260030217DEE59620E7FB759691E51B
:101710009620E7FB900CD8E597F0E020E003021755
:10172000DE7440F0C3900F29E09440900F28E094BD
:1017300000403C900F1BE0FBA3E0FAA3E0F97D40E2
:101740007C007F20126C8C900F1CE475F04012011D
:10175000F3900F29E024C0F0900F28E034FFF090C0
:101760000F27E02440F0900F26E03400F0801C901A
:101770000F28E0FCA3E0FD900F1B7F20126C8490EB
:101780000CD8E04408F0E4900F2AF0900F24E0FE1B
:10179000A3E0FFA3E0B50611A3E0B5070C900CD8B9
:1017A000E04408F0E4900F2AF0900F2AE0701990BE
:1017B0000F1FE0B40912900F1BE0FBA3E0FAA3E0B7
:1017C000F912015EFF126D42900F2AE06404600579
:1017D000E59620E7FB759611900CD8E0F5972290DE
:1017E0000C6AEFF0A3E0FCA3E0FDA3E0FEA3E0FFA2
:1017F000900B551203BDE4FF127340900C72EFF092
:1018000054FEFDE4FF1274C6900C6AE06416706D1D
:101810007F161270BB900C71E0547024F06020248D
:10182000D0602724F0602E24F0603524F0603C2442
:10183000707043900C737401F0A374F4F0803E90C8
:101840000C73E4F0A374FAF08033900C73E4F0A30B
:1018500074C8F08028900C73E4F0A37464F0801DC9
:10186000900C73E4F0A37432F08012900C73E4F0E7
:10187000A37419F08007E4900C73F0A3F0900C733C
:10188000E0FEA3E0FBAA06E4F9F8900C6BE0FCA3F1
:10189000E0FDA3E0FEA3E0FF1202F4900C7B120334
:1018A000BD900C7BE0FCA3E0FDA3E0FEA3E0FF788D
:1018B00006120397EE543FFE900C75EEF0A3EFF086
:1018C000900C75E0FCA3E0FDAE047806C333CE3384
:1018D000CED8F92DFFEC3EFE900C77F0A3EFF0E4AC
:1018E000FCFD900C7BE0F8A3E0F9A3E0FAA3E0FB99
:1018F000D3120386401C900C78E02441F0900C77C2
:10190000E03400F0900C76E004F07006900C75E086
:1019100004F0900C7BA3A3E0FEA3E0FFC3900C783F
:10192000E09FF0900C77E09EF0900C75E0FEA3E055
:10193000FBAA06C3900C78E09421900C77E0940009
:10194000401C900C76E024FFF0900C75E034FFF022
:10195000900C78E024DFF0900C77E034FFF0C39037
:101960000C78E09420900C77E094004011EB1B7011
:10197000011AA3E024E0F0900C77E034FFF0900C23
:1019800077E0FEA3E0FFC39420EE940050A5EF940F
:1019900010EE94004010E024E0F0900C77E034FF6B
:1019A000F0EB1B70011A900C77E0FEA3E0FFC390F0
:1019B0000C76E09FFF900C75E09E900C79F0A3EF01
:1019C000F0900C78E02BFF900C77E03AAD07FC909C
:1019D0000C6AE064167047EDAE047806CEC313CEF1
:1019E00013D8F9540FFF900C71E054F04FF0900CA5
:1019F00079E0FAA3E0FBEA5403FFAE05EE25E0250B
:101A0000E054FC4F900C70F0900C6FEBF07B017A7F
:101A10000C796F900CBA7403F07F16126B03900B65
:101A200054E07003021AD57F121270BB900C71E063
:101A300054FEF0900C70E0543FF04440F07B017A8B
:101A40000C796F900CBA7403F07F12126B037B0158
:101A50007A0C796F7D037F141270C3900C70E04490
:101A600008126AF47F017E001276417F10127340E3
:101A7000EF5407900C7FF0900C70E054F7126AF46A
:101A8000900C7FE0FFD394014005EF94064046E4BC
:101A9000900C75F0A3F0900C76E004F07006900CBA
:101AA00075E004F0900C70E0547F126AF4900C70B2
:101AB000E04480126AF47F0A7E001276417F0E12A3
:101AC0007340EF20E10FC3900C76E09403900C7507
:101AD000E0940040C1900C72E0FDE4FF0274C690F7
:101AE0000C7BEBF0A3EAF0A3E9F0E4900C89F09012
:101AF0000B53E0547FF07F8F1275FC1278E67D4027
:101B00007F1A1274C67D3F7F0D1274C67F807E00DF
:101B10001269B97F8F1275FCE4900B52F0A3F07F2D
:101B20001BFE1269B9900B53E054176003021C1A94
:101B3000900B53E020E303021DA47B017A0E79F69B
:101B40007F011278A7900EF6E054F81313543FFF6C
:101B50007E00900C7FEEF0A3EFF0D39420EE940083
:101B60004009900C7FE4F0A37420F0900C7FA3E078
:101B7000FF900C7BE0FBA3E0FAA3E02424F9E43A15
:101B8000FAEF120199900C80E02404F0900C7FE0B1
:101B90003400F0E0FEA3E07803C333CE33CED8F9AF
:101BA000F0EE900C7FF0E0FCA3E0FDEC5403444029
:101BB000900C83F0EDA3F0900C7FE0FEA3E078039F
:101BC000CEC313CE13D8F9F0EE900C7FF07B017AE0
:101BD0000C7983900CBA7402F07F1A126B03E490B4
:101BE0000B52F0A3F07B01900C8604F0A3740EF06E
:101BF000A374F7F0900C80E024FF8058C3900C8011
:101C0000E09412900C7FE0940040537F067E801297
:101C100069B9900B53E054066009900C8974FFF089
:101C2000021DA47F1C127340900C7EEFF0900B52AB
:101C3000E0547FF0900C86E0FBA3E0FAA3E0F97F8C
:101C4000121278A7900C87E475F0121201F3900C31
:101C500080E024EEF0900C7FE034FFF0809E7F4027
:101C60007E001269B9900B53E054157007900C81F7
:101C700004F08005E4900C81F07F9F1275FC7F1CBE
:101C8000127340EF541F900C7EF06054E0FFFDC3D0
:101C9000900C80E09DF0900C7FE09400F0900C861A
:101CA000E0FBA3E0FAA3E0F91278A7E4900C82F03D
:101CB000FF900C7BE0FBA3E0FAA3E02424F9E43AD4
:101CC000FA12015EFEEFC39E501674F82FF582E4FF
:101CD000340EF583E07006900C82E004F00F80D1A2
:101CE0007D377F0D1274C67F807E001269B97F8FA9
:101CF0001275FC7D207F1B1274C6E4900B52F0A37A
:101D0000F07F5FFE1269B97F1C127340EF541FFF12
:101D10007003021DA47B017A0F79181278A7900C2A
:101D20007BE0FBA3E0FAA3E02424F9E43AFA1201F1
:101D30005EFD900C8E7401F0A3740EF0A374F6F0A7
:101D4000A37401F0A3740EF0A374F8F0A37401F06F
:101D5000A3740FF0A37418F0900C7BA3E0FAA3E037
:101D6000F9124B0F7F0F127340900C7BE0FBA3E046
:101D7000FAA3E02427F9E43AFAEF120199900C81D2
:101D8000E0701B900C7BE0FBA3E0FAA3E02424F9B5
:101D9000E43AFA12015EFF900C82E0B50706900C5F
:101DA000897401F0E4FD7F1A1274C6900C89E0FF7B
:101DB00022900C5B1203BD12781F7F017E00127609
:101DC00041900C5F7455F0A374AAF0E4A3F0A374DF
:101DD000FFF07B017A0C795F900CBA7404F07F16E7
:101DE000126B037E007F047D007B017A0C795F1209
:101DF00005CC7B017A0C795F7D047F161270C3904D
:101E00000C5FE0FFB4550EA3E0B4AA09A3E070058F
:101E1000A3E0F460257BFF7A5B7985900CDCEFF022
:101E2000900C60E0900CDDF0900C61E0900CDEF026
:101E3000900C62E0900CDFF0803CC2A17F017E003C
:101E4000127641D2A17F017E001276417B017A0C8D
:101E5000795F7D047F161270C3900C5FE06455605B
:101E60000FA3E064AA6009A3E06005A3E0B4FF0B40
:101E70007BFF7A5B799A121083803EE4900B52F0DC
:101E8000A3F07D207F0D1274C67D027F1E1274C6E2
:101E90007B017A0C795F900CBA7404F07F1F126B8F
:101EA000037F921275FC7F007E201269B9900B525D
:101EB000E0B4FF0AA3E0B4FF057E007F0122E490B6
:101EC0000B52F0A3F0124CFF7F841275FC1278CCF9
:101ED000EF24C8601C24E8602614602324FC601FE3
:101EE00024257023E4900B54F07BFF7A5B79A98062
:101EF00024900B547401F07BFF7A5B79BF801690BD
:101F00000B547402F080161278CC900CDCEFF07B4E
:101F1000FF7A5B79D51210837E007F0F221274C284
:101F20007D067F011274C67DF07F021274C67D09A2
:101F30007F0A1274C67D087F0A1274C6900C617401
:101F4000E0F0900C6074D8F0900C5F744FF07B015F
:101F50007A0C795F900CBA7403F07F16126B037DD4
:101F6000027F0B1274C6900C5F7401F07403F0A32F
:101F7000743FF0A37420F07B017A0C795F900CBA67
:101F80007403F07F15126B037D377F0D1274C690BA
:101F90000C5F7483F0A304F0A3740AF07A0C795FE9
:101FA000126AF97BFF7A5B79E8121083900C5F74F8
:101FB0000CF0E4A3F0A3F07B017A0C795F900CBAEB
:101FC0007403F07F12126B03E4FF127372900C5BC8
:101FD000E0FCA3E0FDA3E0FEA3E0FF900C6B120386
:101FE000BD7F161217DF7F147E001276417F0E121E
:101FF0007340900C5FEFF020E0057E007F0222909E
:102000000C5FE020E1057E007F0322122BA6900CDE
:1020100063EEF0A3EFF0900C63E0FAA3E0FE3395DB
:10202000E0A3F0A3CEF0900C65E0FCA3E0FDFFAED2
:10203000041201AB900C65EEF0A3EFF0EAFF3395CC
:10204000E0FEA3F0FCA3EFF0FD1201AB900C67EEF5
:10205000F0A3EFF0900C66E02FFF900C65E03EFEE1
:10206000900C63F0A3EFF0D39400EE940240057E51
:10207000007F0E22E4FEFF22900F46EEF0A3EFF069
:10208000A3EBF0A3EAF0A3E9F0E4FFA3F0A3F0FED2
:10209000FD900F47E024F0900F46E034D8C36480F1
:1020A0009480400FA3E024F0F0900F46E034D8F085
:1020B0000F80DE900F47E02418900F46E034FCC3F9
:1020C000648094804014A3E02418F0900F46E0341C
:1020D000FCF0900F4BE004F080D9900F47E0249C77
:1020E000900F46E034FFC3648094804014A3E02442
:1020F0009CF0900F46E034FFF0900F4CE004F0802D
:10210000D9900F47E024F6900F46E034FFC3648077
:102110009480400FA3E024F6F0900F46E034FFF0E7
:102120000E80DE900F47E024FF900F46E034FFC39F
:1021300064809480400FA3E024FFF0900F46E034C9
:10214000FFF00D80DEEF70030221D22430FF900FEC
:1021500048E0FBA3E0FAA3E0F9EF120199900F4BDE
:10216000E02430FF900F48E0FBA3E0FAA3E0240155
:10217000F9E43AFAEF120199900F4CE02430FF9005
:102180000F48E0FBA3E0FAA3E02402F9E43AFAEFF7
:10219000120199EE2430FF900F48E0FBA3E0FAA370
:1021A000E02403F9E43AFAEF120199ED2430FF90AC
:1021B0000F48E0FBA3E0FAA3E02404F9E43AFAEFC5
:1021C000120199900F48E0FBA3E0FAA3E024050276
:1021D0002305900F4BE0606C2430FF900F48E0FB2C
:1021E000A3E0FAA3E0F9EF120199900F4CE024303C
:1021F000FF900F48E0FBA3E0FAA3E02401F9E43AE2
:10220000FAEF120199EE2430FF900F48E0FBA3E0B3
:10221000FAA3E02402F9E43AFAEF120199ED24302E
:10222000FF900F48E0FBA3E0FAA3E02403F9E43AAF
:10223000FAEF120199900F48E0FBA3E0FAA3E02423
:1022400004022305900F4CE060502430FF900F48AB
:10225000E0FBA3E0FAA3E0F9EF120199EE2430FFCE
:10226000900F48E0FBA3E0FAA3E02401F9E43AFA76
:10227000EF120199ED2430FF900F48E0FBA3E0FA44
:10228000A3E02402F9E43AFAEF120199900F48E032
:10229000FBA3E0FAA3E02403806BEE60382430FF58
:1022A000900F48E0FBA3E0FAA3E0F9EF120199EDEB
:1022B0002430FF900F48E0FBA3E0FAA3E02401F9EB
:1022C000E43AFAEF120199900F48E0FBA3E0FAA379
:1022D000E024028030ED60112430FF900F48E0FBD5
:1022E000A3E0FAA3E0F9EF800D900F48E0FBA3E034
:1022F000FAA3E0F97430120199900F48E0FBA3E0D3
:10230000FAA3E02401F9E43AFAE412019922900CCC
:1023100061EBF0A3EAF0A3E9F0A3EDF0E4900C6D1B
:10232000F0A3F0A3F0A3F0900C73F0A37403F0E417
:10233000900B52F0A3F07F8F1275FCE4900C73F0B9
:10234000900C64E0FF900C73E0C39F504D900C61C3
:10235000E0FBA3E0FAA3E0F9900C73E0FF75F0282E
:10236000A4F582E92582F9EA35F0FAE4F5F01202E3
:102370004AEF75F028A4FF900C61E0FBA3E0FAA3FC
:10238000E02FF9EA35F0FAE92424F9E43AFAE41204
:102390000199900C73E004F080A6E4900B52F0A336
:1023A000F0900C65E0FBA3E0FAA3E0F9A3E0FD12D6
:1023B0002F457F2C7E0112784DE4900B52F0A3F054
:1023C000900C69E0FF12694EE4900C6FF0A3F07F6F
:1023D00001FEFDFC900C69E0F9F81203AA900C7163
:1023E000EEF0A3EFF0900C64E0FD900C6DE0FEA326
:1023F000E0FFC39DEE940040030224D27C007D28C0
:102400001201AB900C61E0FBA3E0FAA3E02FF9EA24
:102410003EFA126C22EF14601424027067900C7064
:10242000E004F0705F900C6FE004F08057900C684F
:10243000E0FF7E00C006C007900C6DE0FEA3E0FF49
:102440007C007D281201AB900C61E0FBA3E0FAA3B5
:10245000E02FF9EA3EFAE92404F9E43AA801FCADD8
:1024600003900C65E0FBA3E0FAA3E0F9D007D006E7
:102470001205A8EF700E900C6EE004F07006900C40
:102480006DE004F0900C72E024FFF0900C71E034E9
:10249000FFF0E4900B52F0A3F0900C6AA3E0FAA3D3
:1024A000E0F91203EF900C75EFF0900C71E0700200
:1024B000A3E0600B900C75E060057F991275FC90AD
:1024C0000C71E07002A3E06009900C75E0600302FB
:1024D00023E5900C74E014F0900C6FE07002A3E020
:1024E000607DE47F01FEFDFC900C69E0F9F81203C9
:1024F000AAE47B04FAF9F81202F4A804A905AA06D2
:10250000AB07900C6FE0FEA3E0FFE4FCFDD31203E9
:1025100086500A900C69E004F07F9A803DE47F01C8
:10252000FEFDFC900C69E0F9F81203AAE47B08FABE
:10253000F9F81202F4A804A905AA06AB07900C6FDB
:10254000E0FEA3E0FFE4FCFDD3120386400A900CFA
:1025500069E014F07F9C80027F9B1275FC8005E48B
:10256000900C74F0900C64E0FFC3900C6EE09F90B0
:102570000C6DE094005018900C74E06012900C6A9E
:10258000A3E0FAA3E0F91203EFEF60030223C8907F
:102590000C6DE0FEA3E0FF22900C5DEBF0A3EAF0EF
:1025A000A3E9F0A3EDF0E4900C66F0900C79740AC6
:1025B000F0A37432F0127103C292D2931278D290C7
:1025C0000C61E0FFA3E0FBA3E0FAA3E0F9A3E09035
:1025D0000C82F0124A14D292D2937F047E001276BB
:1025E000411277B2125C26900C77EFF0706D7B0190
:1025F000900C8204F0A3740CF0A3746FF0A3740821
:10260000F0124113900C5DE0FBA3E0FAA3E0242458
:10261000F9E43AFA7408120199900C5DE0FBA3E02A
:10262000FAA3E02404F9E43AFA900CDCEBF0A3EA14
:10263000F0A3E9F0900C5DA3E0FAA3E02424F9E410
:102640003AFA12015E900CDFF07B017A0C79671286
:102650007190900C667401F00227E3900C77E0B45F
:10266000FD08E4900C66F00227E3900C7B74FFF009
:10267000A37478F0A374DCF0900C787402F0900CE2
:1026800060E070030227E3900C79E0FF900C78E0A3
:10269000C39F40030227E3900C7AE0FF14F0EF7031
:1026A000030227E3127103C292D293900C7BA3E042
:1026B000FAA3E0F91203EFD292D2937F047E0012C4
:1026C00076411277B2125C26900C77EFF0601424FA
:1026D0000370030227882402600302279F900C7B6B
:1026E0000227CF900C827401F0A3740CF0A3746FD6
:1026F000F0A37408F07B01124113900C66E075F0B2
:1027000028A4FFAEF0900C5DE0FBA3E0FAA3E02F5D
:10271000F9EA3EFAE92424F9E43AFA740812019934
:10272000900C5DE0FBA3E0FAA3E02FF9EA3EFAE9A2
:102730002404F9E43AFA900CDCEBF0A3EAF0A3E904
:10274000F0900C5DA3E0FAA3E02FF9EA3EFAE92449
:1027500024F9E43AFA12015E900CDFF07B017A0C66
:102760007967127190900C66E004F0900C60E014B0
:10277000F0900C78E014F0900C7B74FFF0A3747868
:10278000F0A374D7F002267E900C7B74FFF0A37444
:1027900078F0A374D7F0900C78E014F002267E90C5
:1027A0000C7BE0FBA3E0FAA3E0F9EB8A838982F4D7
:1027B000700A74266582700474006583900C7B60D7
:1027C0000E74FFF0A37400F0A37426F002267E744A
:1027D000FFF0A37478F0A374DCF0900C78E004F0C0
:1027E00002267E900C66E0FF22011000010A000123
:1027F0001101500F2DBFAFA7A3A1A0B0B8BCBE411F
:10280000888A642082480DB6FFFFFFFFFFFFFFFFAD
:1028100060400D33000000000000000000000000D8
:1028200000000000000000000000000000000000A8
:102830000000000000000000000000000000000098
:102840000000000000000000000000000000000088
:1028500000000000490F3DFF7E9CFF7EA1FF7EAD82
:10286000430F2A0003034C0E7F05FF746C00000029
:102870000000000000500E6A02FF77080000000010
:102880000000000000000000410E7A00440B3C06EE
:10289000010001410B4304410B4D03410B4C3244F9
:1028A0000B48000DC65E440003000E2612420B3595
:1028B0000000420B130190420B4100004100000058
:1028C0004100010041000200410B5100410B4E004C
:1028D000420B52000060FC0B59000001020304058A
:1028E000060708090A0B0C0D0E0F10111213141510
:1028F000161718191A1B1C1D1E1F20212223242500
:10290000262728292A2B2C2D2E2F303132333435EF
:10291000363738393A3B3C3D3E3F404142434445DF
:10292000464748494A4B4C4D4E4F505152535455CF
:10293000565758595A5B5C5D5E5F606162636465BF
:10294000666768696A6B6C6D6E6F707172737475AF
:10295000767778797A7B7C7D7E7F8081828384859F
:10296000868788898A8B8C8D8E8F9091929394958F
:10297000969798999A9B9C9D9E9FA0A1A2A3A4A57F
:10298000A6A7A8A9AAABACADAEAFB0B1B2B3B4B56F
:10299000B6B7B8B9BABBBCBDBEBFC0C1C2C3C4C55F
:1029A000C6C7C8C9CACBCCCDCECFD0D1D2D3D4D54F
:1029B000D6D7D8D9DADBDCDDDEDFE0E1E2E3E4E53F
:1029C000E6E7E8E9EAEBECEDEEEFF0F1F2F3F4F52F
:1029D000F6F7F8F9FA00E4900C5BF0900E7B744087
:1029E000F0A37401F0A3740DF0A37475F0900D754D
:1029F0007444F0A37440F0900E28E0640170527F9C
:102A0000011271D112375FE4900002F0900B11F0C7
:102A1000A3F0EF70377B01900C6504F0A3740BF00A
:102A2000A37415F0E4A3F0900B43E0900C69F0A3BD
:102A300074FFF0A37475F0A3743FF07A0179117DEF
:102A40004012230E900B11EEF0A3EFF0E4FF12738F
:102A5000D9900002E0FFD3900B12E09F900B11E0A1
:102A600094005003022B7A900002E0FD75F028A438
:102A70002435F582E5F03401F583E0FE240A900D5B
:102A800076F0EE2402900D7CF075F028EDA424136E
:102A9000F582E5F03401F583E0900D7DF0900002C1
:102AA000E075F028A42414F582E5F03401F583E004
:102AB000900D7EF0EF75F028A42415F9740135F01F
:102AC000FA7B01C003900CDCEBF0A3740DF0A3744F
:102AD0007FF0900002E075F028A42435F582E5F03F
:102AE0003401F583E0900CDFF0D003127190900078
:102AF00002E075F028A42438F582E5F03401F5836E
:102B0000E0900D78F0900B37E0FEA3E07802C3333D
:102B1000CE33CED8F9FBAA062408F58274003AF524
:102B200083A3A3A3E0FF900D79EFF074082BF58247
:102B300074003AF583E0FCA3E0FDA3E0FEA3E0FF10
:102B40007808120397900D7AEFF0900B37E0FEA310
:102B5000E07802C333CE33CED8F92408F58274006E
:102B60003EF583E0FCA3E0FDA3E0FEA3E0FF7810C8
:102B7000120397900D7BEFF0800B900D767405F0AB
:102B8000E4900D79F0900B11E0FEA3E0FF4E600A97
:102B9000900002E0FEC3EF9E8001E4900D77F0907C
:102BA0000002E004F022E4FF127340900C73EFF097
:102BB0007B017A0C796F7D037F141270C3900C6FC8
:102BC000E0900C72F054CF900C6FF07B017A0C798E
:102BD0006F126AFB1274C27F961275FC7F017E0031
:102BE0001276417F971275FC7D017F111274C67FAA
:102BF000027E001276417F871275FC7F147E0012E0
:102C0000784D7F19127340900C6DEFF05480FF33B4
:102C100095E04F6006E0547FFF8009900C6DE05412
:102C20007FF404FF900C6DEFF07D027F111274C6EB
:102C30007F027E001276417F871275FC7F147E0032
:102C400012784D7F19127340900C6EEFF05480FF94
:102C50003395E04F6006E0547FFF8009900C6EE0F2
:102C6000547FF404FF900C6EEFF07D03E4FF1274C8
:102C7000C67F961275FC7F017E001276417F971207
:102C800075FC7D017F111274C67F027E00127641B1
:102C90007F871275FC7F147E0012784D7F191273A6
:102CA00040900C6CEFF05480FF3395E04F6006E0ED
:102CB000547FFF8009900C6CE0547FF404FF900C6B
:102CC0006CEFF0A3E0FD3395E0FCEF3395E0FEC33D
:102CD000EF9DFFEE9C900C6AF0A3EFF07D027F1158
:102CE0001274C67F027E001276417F871275FC7FC8
:102CF000147E0012784D7F19127340900C6CEFF027
:102D00007F961275FC900C6CE0FF5480FD3395E0CB
:102D10004D6006EF547FFF8009900C6CE0547FF407
:102D200004FF900C6CEFF0900C6EE0FEC3EF9EFF82
:102D3000900C6CF0EFFE900C6BE0FDEDFF900C6AD8
:102D4000EEF0A3EFF07B017A0C796F7D037F141214
:102D500070C3900C72E0900C6FF07B017A0C796F6D
:102D6000126AFB900C73E0FDE4FF1274C6900C6ACB
:102D7000E0FEA3E0FF22FDF0900C86E0FF3395E03B
:102D8000FEEF25E0FFEE33FE748B2FF9740E3EFA52
:102D90007B01900C99EBF0A3EAF0A3E9F0900C9979
:102DA000E0FBA3E0FAA3E0F9E4120199900C99E0AA
:102DB000FBA3E0FAA3E02402F9E43AFAE412019951
:102DC000900C99E0FBA3E0FAA3E02401F9E43AFABD
:102DD0007408120199900C99E0FBA3E0FAA3E02497
:102DE00003F9E43AFA7408120199ED900C9930E76E
:102DF0000FE0FBA3E0FAA3E0F912015E4480800D2E
:102E0000E0FBA3E0FAA3E0F912015E44401201994D
:102E1000ED900C9930E60FE0FBA3E0FAA3E0F91285
:102E2000015E4420800DE0FBA3E0FAA3E0F912016B
:102E30005E4410120199ED900C9930E50FE0FBA370
:102E4000E0FAA3E0F912015E4408800DE0FBA3E084
:102E5000FAA3E0F912015E4404120199ED900C9975
:102E600030E40FE0FBA3E0FAA3E0F912015E4402B4
:102E7000800DE0FBA3E0FAA3E0F912015E44011229
:102E80000199ED900C9930E314E0FBA3E0FAA3E084
:102E90002402F9E43AFA12015E44808012E0FBA3B6
:102EA000E0FAA3E02402F9E43AFA12015E44401287
:102EB0000199ED900C9930E214E0FBA3E0FAA3E055
:102EC0002402F9E43AFA12015E44208012E0FBA3E6
:102ED000E0FAA3E02402F9E43AFA12015E44101287
:102EE0000199ED900C9930E114E0FBA3E0FAA3E026
:102EF0002402F9E43AFA12015E44088012E0FBA3CE
:102F0000E0FAA3E02402F9E43AFA12015E44041262
:102F10000199ED900C9930E014E0FBA3E0FAA3E0F6
:102F20002402F9E43AFA12015E44028012E0FBA3A3
:102F3000E0FAA3E02402F9E43AFA12015E44011235
:102F400001997F0222900C76EBF0A3EAF0A3E9F05E
:102F5000A3EDF0A37412F07F8F1275FC784D768F7D
:102F6000087690900C79E0FD2403FFE433FEEF78BF
:102F700004CEA2E713CE13D8F87821F6ED2403543B
:102F80000FC454F0440B08F6900C79E033333354FB
:102F9000F8FFF0900EF3E025E0540E44A008F60888
:102FA0007612900C79E0FEC4540F08F6EEC454F08B
:102FB00008F67E05EFC39408403A74212EF8C0004D
:102FC000E6FD900C76E0FBA3E0FAA3E0F912015EC7
:102FD000FCC4540F4DD000F60EECC454F0FD742127
:102FE0002EF8A60574F82FFF900C77E475F0011207
:102FF00001F380C074212EF8E6F6900C79E0FF13FF
:103000001313541FF0E02406F0900C7BE4F0A3743B
:1030100000F0A37421F0900C79E0D3941A500302CD
:1030200030DB900B52E054BFF0900C83741DF09095
:103030000C7BE0F9A3E0FAA3E0900C84C9F0A3EACA
:10304000F0A3E9F0A3741AF07B007A00794E7D01B9
:10305000126CE4900C79E024E6F0900C7CE475F0BE
:103060001A804E900C7AE0FF900C79E0D39F404696
:103070007D0F7C007F007E4012666C900B52E05406
:10308000BFF0900C7BE0FBA3E0FAA3E0F9900C7A90
:10309000E0900CBAF07F1F126B03900C79E0FFA355
:1030A000E0FEC3EF9E900C79F0EEFF900C7CE48F75
:1030B000F01201F380AD7D0F7C007F007E40126630
:1030C0006C900C7BE0FBA3E0FAA3E0F9900C79E0B4
:1030D000900CBAF07F1F126B03802E900C83741D2E
:1030E000F0900C7BE0F9A3E0FAA3E0900C84C9F027
:1030F000A3EAF0A3E9F0900C79E0900C87F07B0054
:103100007A00794E7D01126CE47D0F7C007F807E19
:103110000002666C900C5DEBF0A3EAF0A3E9F0A36B
:10312000EDF0900C68740DF0E4900C67F0900C6476
:10313000E0FF14F0EF70030232A7900C67E0600329
:103140000232A7127103C292D293D2937F017E0002
:103150001276411254D1900C65EFF03395E0FEEFFA
:1031600025E0FFEE33FE748B2FF9740E3EFA7B01DF
:10317000900C68E0FD122D92900C65E02FF0900C01
:1031800068E0A3F0E4900C66F0900C5DE0FBA3E037
:10319000FAA3E0F9900C66E0FFFD3395E0FCE92D21
:1031A000F9EA3CFA12015EFEEF3395E0FC746A2DF9
:1031B000F582740C3CF583EEF0900C65E0FF3395DE
:1031C000E0FEEF25E0FFEE33FE748B2FF9740E3E28
:1031D000FA7B01746A2DF582740C3CF583E0FD12D4
:1031E0002D92900C65E02FF0A3E004F0E0C3648022
:1031F00094884095900C60E0FD900C72F0900C6506
:10320000122D7B900C65E02FF0900C60E004F0A391
:10321000E0FBA3E0FAA3E0F912015EFD900C73F06D
:10322000900C65122D7B900C65E02FF0900C62E401
:1032300075F0011201F37B017A0C79697D0B7C003A
:10324000126058900C65126D9E900C65E02FF07B1B
:10325000017A0E798BE0FD3395E0FC127497D293DE
:10326000D292D2937F047E001276411277B27B0114
:103270007A0C79747D01125C2E900C67EFF0700E61
:10328000900C74E07FFC7001FF900C67EFF01271FE
:1032900003C292D293D2937F0F7E001276411272B4
:1032A000101277B202312D900C67E0FF22900C5E75
:1032B000EBF0A3EAF0A3E9F0900EF57401F078F1D9
:1032C0007C0EFD900C5EE0FBA3E0FAA3E0F97E002B
:1032D0007F04120116900EF2E07005900EF404F0D7
:1032E000900C5EE0FBA3E0FAA3E0F912015E70032C
:1032F0000233BC24FA700302339A24FE607814600F
:103300005224FD602A24FD6003023440E4900C61E5
:10331000F0A374F0F0A374F2F0A3744DF0A3740161
:10332000F0A37404F0E4A3F0A37407F00233E39075
:103330000C617401F0A374F0F0A374C2F0A3749B49
:10334000F0A37402F0A37406F0E4A3F0A37427F0D2
:103350000233E3900C617401F0A374F0F0A3749253
:10336000F0A37441F0A37403F0A37405F0A314F068
:10337000A37437F0806D900C617402F0A374F0F0C8
:10338000A37482F0A374E8F0A37403F0A37406F0AE
:10339000A37404F0A3743BF08049900C617402F0B4
:1033A000A374F0F0A37462F0A37435F0A37405F075
:1033B000A37407F0A3F0A3743FF08027900C61740E
:1033C00002F0A374F0F0A37402F0A374D0F0A3741D
:1033D00007F0A3741BF0A37407F0A374FFF0E4904C
:1033E0000EF5F0900EF2E025E025E0FF900C61E094
:1033F00054F34FF0900EF4E07F0060027F01EF2560
:10340000E0FF900C63E054FD4FF07B017A0C796192
:10341000900CBA7404F07F01126B037F05127340A5
:10342000EF54F0FF900C65E04FFD7F051274C67BF2
:10343000017A0C7966900CBA7403F07F07126B0363
:1034400022900C6CEBF0A3EAF0A3E9F0EEC313FEBC
:10345000EF13FF900C76EEF0A3EFF04E7007900C98
:1034600076F0A304F0E4FF127340900C72EFF012B8
:1034700074C27F09127340900C75EFF07DFF7F09D5
:103480001274C6900C72E020E1077F0A7E0012766B
:1034900041E4900C78F0900C7674FFF5F01202097C
:1034A00045F06048127568900C73EFF0E0FFC4546B
:1034B0000FFEEF540F2EFF900C79F0900C78E0FD8A
:1034C0003395E0FCD3EF9DEC6480F874809840C69F
:1034D000A3E0900C78F0900C73E0FF900C6CE0FB94
:1034E000A3E0FAA3E0F9EF12019980AA900C78E02A
:1034F000FF701F900C6FE0FBA3E0FAA3E0F974806B
:10350000120199900C6CE0FBA3E0FAA3E0F9E4024D
:1035100035ABEF7803A2E713D8FBFF900C78E02FD0
:10352000F07F0A127340900C74EFF07F0512734025
:10353000900C74E0FE30E211900C78E024B5F0EECF
:1035400030E023E02405F0801D900C78E024B9F0F1
:10355000EE30E104E024F6F0900C74E030E00790E7
:103560000C78E02408F0EF30E71C900C78E0FF9036
:103570000C74E0C41313540375F003A4FEC3EF9E50
:10358000900C78F08014900C74E0C41313540375FD
:10359000F003A4FF900C78E02FF0900C78E0FF90FF
:1035A0000C6FE0FBA3E0FAA3E0F9EF120199900C95
:1035B00075E0FD7F091274C6900C72E0FDE4FF1205
:1035C00074C6900C72E030E0077F027E00127641F4
:1035D00022900C61EBF0A3EAF0A3E9F0E4900C6A0E
:1035E000F0A3F0784D768F0876917821F60876551D
:1035F0000876C2AF05EFC4333354C0FF08F6900C11
:1036000065E0FE1313543F4FF6EEC4333354C0FF4E
:1036100008F6A3E0FE1313543F4FF6EEC4333354C1
:10362000C0FF08F6E92425F9E43AFA12015EFE1318
:1036300013543F4FF6EEC4333354C0FF08F6900CDA
:1036400061E0FBA3E0FAA3E02426F9E43AFA1201D0
:103650005EFE1313543F4FF6EEC4333354C008F6E6
:10366000E4900B52F0A3F07F8F1275FC900C8374E2
:103670001DF0A3E4F0A37400F0A37421F0A3740878
:10368000F07B007A00794E7D01126CE47F807E0031
:103690001269B9E4900B52F0A3F07F8F1275FC7F92
:1036A0005E7E801269B9900B53E030E333900C6773
:1036B000E0FBA3E0FAA3E0F97F011278A7900C6782
:1036C000E0FBA3E0FAA3E0F912015E448012019945
:1036D000900C67E0FBA3E0FAA3E0F912015EFF2281
:1036E000900B53E0541F600F7F1C127340EF541F68
:1036F000900C6BF07F0822900B52E030E731900C79
:1037000067E0FBA3E0FAA3E0F97F121278A7900C20
:1037100068E475F0121201F3900C6AE02412F09044
:103720000B52E0547FF07F5E7E801269B980C8E45E
:10373000900B52F0A3F07F1C127340EF541FFF90C8
:103740000C6BF0900C67E0FBA3E0FAA3E0F91278B1
:10375000A7900C6BE0FF900C6AE02FF07F002290A6
:103760000B13E0FCA3E0FD24F0FBEC34FFFAD3EBF9
:1037700094E8EA9403401BED2410FFE43CFEEF784C
:1037800006CEC313CE13D8F9FF7C007D301201ABF7
:1037900080167C007D30AF03AE021201ABEF7806DD
:1037A000CEC313CE13D8F9FF900B39EEF0A3EFF090
:1037B000E4FF1273D9900B35E0FEA3E0FFD394141D
:1037C000EE9400400BEF24ECFFEE34FFFE12764146
:1037D000900007E070037F0A22900B37A3E0900C63
:1037E00062F0900B41E0FEA3E0FF900C6F7401F0DB
:1037F000A3740CF0A37463F07B017A0C7964123427
:1038000041E4900C61F0900007E0FF900B37E47505
:10381000F0011201F3FCC3E5F09FEC94004007E4D3
:10382000900B37F0A3F0900B37E0FEA3E07802C3D3
:1038300033CE33CED8F92408F58274003EF583E008
:10384000FCA3E0FDA3E0FEA3E0FF900C6B1203BD20
:103850007F161217DF900B41E0FEA3E0FF900C6F84
:103860007401F0A3740CF0A37463F07B017A0C79FB
:1038700064123441900B37E0FEA3E024DCF582743F
:10388000003EF583E0FF900C63E0FED3EF6480F828
:10389000EE648098400F900C61E004F0E0C3943532
:1038A0005003023806900B37E0FEA3E024DCF582DB
:1038B00074003EF583E0FF900C63E0FED3EF64807C
:1038C000F8EE64809850171275D8E4900B3BF07FA7
:1038D000011273D97F027E001276417F0022900B85
:1038E0003B7401F0E4FF1273D97F0A22900F20E0AD
:1038F00024DF70030239DD1470030239FB2421B484
:1039000005004003023A1590391575F003A4C583EC
:1039100025F0C5837302392402393702395D023933
:103920008C0239A6900F1B74FFF0A3747CF0A37473
:103930001FF0907C1F8066900F1B74FFF0A3747CB7
:10394000F0A37431F0907C34E493FE907C33E493E4
:103950007C002400FFEC3E900F280239F5900F21E7
:10396000E075F003A4243DF582E5F0340FF583E023
:10397000FBA3E0FAA3E0F9900F1BEBF0A3EAF0A39E
:10398000E9F012015EFF900F28E48069900F1B742C
:10399000FFF0A3747CF0A3743AF0907C3AE493FFB8
:1039A000900F28E4804F900F21E0FF64817066EF54
:1039B000900F1BB4811074FFF0A3747CF0A3744CBF
:1039C000F0907C4C800E74FFF0A3747CF0A37453D1
:1039D000F0907C53E493FF900F28E48018900F1B25
:1039E00074FFF0A3747CF0A37443F0907C43E493E1
:1039F000FF900F28E4F0A3EFF0801D900F1B74FFE1
:103A0000F0A3747CF0A3745AF0900F287402F0A312
:103A10007442F0800312769C900F20E0FF640160F6
:103A200013EF6402600EEF64036009EF6404600446
:103A3000EFB40523900F25E0FFD3900F29E09F906E
:103A40000F28E094004010900F24E0700AE0FE90F0
:103A50000F28EEF0A3EFF0900F2AE064046018E561
:103A60009620E7FB759611759740900F2A7401F028
:103A7000E4900F26F0A3F022900C5FEBF0A3EAF0A5
:103A8000A3E9F0E4900C65F0900C5FE0FBA3E0FA92
:103A9000A3E02425F9E43AFA900C7B7401F0A374B6
:103AA0000CF0A37466F0125059EF6008E4900B52CA
:103AB000F0A3F022784D768F087690E47821F6080E
:103AC00076500876C6900C62E0FBA3E0FAA3E0F91A
:103AD00012015EFF900C66E06F08F6E92401F9E43C
:103AE0003AFA12015EFF900C67E06F08F6900C5FE7
:103AF000E0FBA3E0FAA3E02425F9E43AFA12015E20
:103B000008F6900C5FE0FBA3E0FAA3E02426F9E4BA
:103B10003AFA12015E08F67F8F1275FCE4900B52A0
:103B2000F0A3F0900C83741DF0A3E4F0A37400F0F4
:103B3000A37421F0A37407F07B007A00794E7D0115
:103B4000126CE4E4900B52F0A3F07F5FFE1269B9AF
:103B5000900B53E020E0767F1C127340EF540FFF70
:103B6000C3940340027F037B017A0C79681278A723
:103B7000900C5FE0FBA3E0FAA3E02426F9E43AFA14
:103B800012015EFF900C69E06F7038900C5FA3E04B
:103B9000FAA3E02425F9E43AFA12015EFF900C68DA
:103BA000E0B5071F7F8F1275FCE4900B52F0A3F075
:103BB000900C6375F0021201F3900C65E0B40115EE
:103BC0007F0022E4900B52F0A3F07F0222900C655C
:103BD0007402F0FF22E4900B52F0A3F0900C65E029
:103BE00004F0E0C394025003023A887F00221237A7
:103BF0005F900C5EEFF06003023D0A12686D900B5F
:103C000011E07002A3E07009900C5E7409F0023DAF
:103C10000A900E2AE0700CA3E07008A3E07004A3E1
:103C2000E06026900C627401F0A3740EF0A3742A75
:103C3000F0900B44E0FBA3E0FAA3E0F9123A78908D
:103C40000C5EEFF06003023D0A900E28E0FFB40125
:103C5000057402F0800AEFB40206900E287401F099
:103C6000E4900C5BF0A3F0A3F0900E29E0FD70103F
:103C7000900C5B74C0F0900E28E0FEC45430802B92
:103C8000EDB40113900C5B7430F0900E28E0FF252A
:103C9000E025E0540C8014900E29E0FDB40212904F
:103CA0000C5B740CF0900E28E05403900C5CF080D8
:103CB00038EDB40312900C5B7403F0900E28E0FF13
:103CC000C4333354C08015900E29E0B40414900C12
:103CD0005C74C0F0900E28E0FFC45430900C5DF08E
:103CE0008007E4900C5BF0A3F0900C627401F0A3E9
:103CF000740CF0A3745BF0900B44E0FBA3E0FAA318
:103D0000E0F9124F94900C5EEFF0E4FF1273D9903B
:103D10000D75743CF0A37404F0900C5EE0900D7788
:103D2000F0900E7CE0FBA3E0FAA3E02401F9E43A72
:103D3000FA12015E900E7BF0A37401F0A3740DF0F3
:103D4000A37475F07F3C024DEA12375F900C5BEF75
:103D5000F06003023E4F12686D900B11E07002A3F9
:103D6000E07009900C5B7409F0023E4F900E2AE05F
:103D70007017A3E07013A3E0700FA3E0700B7BFF3C
:103D80007A6179FD1210838021900C627401F0A396
:103D9000740EF0A3742AF0900B44E0FBA3E0FAA3A6
:103DA000E0F9123A78900C5BEFF0900E28E024FED8
:103DB000602324FA605314606524086003023E4FB8
:103DC000900B44E0FBA3E0FAA3E0F9900E29E0FD9C
:103DD0001256388042900E29E06010900B44E0FBB0
:103DE000A3E0FAA3E0F9125999801C900C5F7401CA
:103DF000F0A3740EF0A3742AF0900B44E0FBA3E050
:103E0000FAA3E0F9124915800E900B44E0FBA3E001
:103E1000FAA3E0F9125A3E900C5BEFF08031900C5F
:103E20005F7401F0A3740EF0A3742EF0900B44E0C5
:103E3000FBA3E0FAA3E0F9124C08900C5BEFF090C2
:103E40000E2EE0900D78F0900E2FE0900D79F0E4BA
:103E5000FF1273D9900D757446F0A37405F0900CA1
:103E60005BE0900D77F0900E7CE0FBA3E0FAA3E01E
:103E70002401F9E43AFA12015E900E7BF0A374017A
:103E8000F0A3740DF0A37475F07F46024DEAE49040
:103E90000C5BF0900E28E0640170527F011271D12A
:103EA00012375FE4900001F0900B11F0A3F0EF7077
:103EB000377B01900C6504F0A3740BF0A37415F02C
:103EC000E4A3F0900B43E0900C69F0A374FFF0A31F
:103ED0007475F0A3743FF07A0179117D4012230EBE
:103EE000900B11EEF0A3EFF0E4FF1273D9900E7C6B
:103EF0007401F0A3740DF0A37475F0900E7B744000
:103F0000F0900D757432F0900B11E0FEA3E0FF4EBF
:103F1000600A900001E0FEC3EF9E8001E4900D77FF
:103F2000F0900001E0FFD3900B12E09F900B11E0A6
:103F300094005003023FC0900001E0FD75F028A4FA
:103F40002435F582E5F03401F583E0FE2406900D7A
:103F500076F0EE2402900D78F075F028EDA424138D
:103F6000F582E5F03401F583E0900D79F0900001E1
:103F7000E075F028A42414F582E5F03401F583E01F
:103F8000900D7AF0EF75F028A42415F9740135F03E
:103F9000FA7B01C003900CDCEBF0A3740DF0A3746A
:103FA0007BF0900001E075F028A42435F582E5F05F
:103FB0003401F583E0900CDFF0D003127190800B98
:103FC000900D767404F0E4900D78F0900001E00418
:103FD000F022900F4DEBF0A3EAF0A3E9F0A3EDF08F
:103FE000E4900F52F07BFF7A5D7987900F51E0905B
:103FF0000CDCF0121083900F4DE0FBA3E0FAA3E07D
:104000002401F9E43AFA12015E900CDCF0900F4DB5
:10401000A3E0FAA3E0F912015E900CDDF07BFF7AD9
:104020005D79921210837BFF7A5D79A3900F50E047
:104030002402900CDCF0121083900F4DE0FBA3E003
:10404000FAA3E02403F9E43AFA12015E900CDCF0E2
:10405000900F4DA3E0FAA3E02402F9E43AFA12012A
:104060005E900CDDF07BFF7A5D79BD1210837BFFE3
:104070007A5D79CB121083900F50E0FF900F52E0E1
:10408000FEC39F5030900F4DE0FBA3E0FAA3E02465
:1040900004F9E43AFAEE7E0029F9EE3AFA12015EEA
:1040A000900CDCF07BFF7A5D797F121083900F52C9
:1040B000E004F080C27BFF7A5D7985121083900F57
:1040C0004DE0FBA3E0FAA3E02424F9E43AFA12015C
:1040D0005E900CDCF07BFF7A5D79D1121083900F3B
:1040E0004DE0FBA3E0FAA3E02425F9E43AFA12013B
:1040F0005E900CDCF0900F4DA3E0FAA3E02426F9CB
:10410000E43AFA12015E900CDDF07BFF7A5D79E70C
:104110000210837A0C7967E4FD900C7EEBF0A3EA41
:10412000F0A3E9F0A3EDF0900C937451F012710339
:10413000C292D293D2937F017E001276411254D163
:10414000900C86EFF03395E0FEEF25E0FFEE33FEB6
:10415000748B2FF9740E3EFA7B01900C93E0FD12E4
:104160002D92900C86E02FF0900C93E0900C88F04C
:10417000E4900C87F0900C7EE0FBA3E0FAA3E0F95A
:10418000900C87E0FFFD3395E0FCE92DF9EA3CFA5D
:1041900012015EFEEF3395E0FC74892DF582740CFC
:1041A0003CF583EEF0900C86E0FF3395E0FEEF25C2
:1041B000E0FFEE33FE748B2FF9740E3EFA7B017430
:1041C000892DF582740C3CF583E0FD122D92900C44
:1041D00086E02FF0A3E004F0E0C36480948840956B
:1041E000900C81E0900C91122D76900C86E02FF0CF
:1041F000900C85E014900C92122D76900C86E02F96
:10420000F07B017A0C79887D0B7C00126058900C51
:1042100086126D9E900C86E02FF07B017A0E798BD2
:10422000E0FD3395E0FC127497D293D292D2939032
:104230000C85E075F004A4FFAEF01276411277B25F
:10424000900C82E0FBA3E0FAA3E0F9A3E0FD125C8E
:104250002E22E4900C5BF0900E28E0640170697FE0
:10426000021271D112375F900C5CEFF0E490000005
:10427000F0126B5B900C5CE06009E4900B11F0A312
:10428000F08032900E29E0900C61F0A37401F0A34D
:10429000740EF0A3742AF0900E32E0900C65F07B5F
:1042A000017A0179117D40122598EF3395E0900B4A
:1042B00011F0A3EFF0E4FF1273D9900B447401F0F6
:1042C000A37401F0A37411F0E4900C5BF0900C5B0C
:1042D000E0FFC3940C501474752FF582E4340DF58F
:1042E00083E4F0900C5BE004F080E2900D75744084
:1042F000F0A3740DF0E4900D78F0900000E0FF75ED
:10430000F028A42435F582E5F03401F583E0900D22
:1043100079F0603AEF75F028A42415F9740135F0AE
:10432000FA7B01C003900CDCEBF0A3740DF0A374D6
:104330007AF0900000E075F028A42435F582E5F0CD
:104340003401F583E0900CDFF0D003127190900BF4
:1043500011E0FEA3E0FF4E600E900000E0FEC3EF10
:104360009E900D77F08009900D767405F0E4A3F02F
:10437000900000E004F0900E7B740DF0A37401F047
:10438000A3740DF0A37475F07F40024DEAE4900C25
:104390005CF0900E2AE0900C5BF012375F900C5CA2
:1043A000EFF0600302448712686D900B11E0700219
:1043B000A3E07009900C5C7409F0024487900C5BD8
:1043C000E060030244557B01900C5D04F0A3740D82
:1043D000F0A37479F0900E29E0900C60F0900C5CE2
:1043E000E0705E900C5BE0C3941E505512753FEF79
:1043F000604F900E28E0FD900C60E0FF04F0900C00
:1044000065EFF0A37401F0900C5DE0F9A3E0FAA36E
:10441000E0900C67C9F0A3EAF0A3E9F0900B44E048
:10442000FBA3E0FAA3E0F91235D1900C5CEFF09019
:104430000C5BE004F0900C5EE475F0021201F38076
:104440009C900C5BE014F0900B3BE0603A900C5CAD
:10445000740AF08032900E28E0FDA3E0900C65F025
:10446000900C5BE0900C66F0A37401F0A3740DF067
:10447000A37479F0900B44E0FBA3E0FAA3E0F912F7
:1044800035D1900C5CEFF0E4FF1273D9900D757488
:1044900038F0900C5CE0900D77F0900C5BE0FD251F
:1044A000E02404900D76F0900D78EDF0900E7B7482
:1044B00040F0A37401F0A3740DF0A37475F07F387D
:1044C000024DEA900C5CEBF0A3EAF0A3E9F0E49073
:1044D0000C63F0900C5CE0FBA3E0FAA3E02425F968
:1044E000E43AFA900C7B7401F0A3740CF0A37464AA
:1044F000F0125059EF600122784D768F900C63E0F6
:10450000FE7003087690EEB40104784E7691E4785C
:1045100021F60876570876C4900C5FE0FBA3E0FA1A
:10452000A3E0F912015EFF900C64E06F08F6E92445
:1045300001F9E43AFA12015EFF900C65E06F08F6AB
:10454000900C5CE0FBA3E0FAA3E02425F9E43AFA3E
:1045500012015EFF131313541FFE900C62E0C4336C
:1045600054E04E08F6900C5CE0FBA3E0FAA3E024D4
:1045700026F9E43AFA12015EFE131313541FFDEFFD
:10458000C43354E04D08F6EEC43354E008F67D36EB
:104590007F0D1274C67F8F1275FCE4900B52F0A34E
:1045A000F0900C83741DF0A3E4F0A37400F0A374E6
:1045B00021F0A37408F07B007A00794E7D01126C23
:1045C000E4900C5C125AE3EF600122900C60E475F9
:1045D000F0021201F3900C63E004F0E0C394025087
:1045E000030244D37F0022900C71EDF0900C6EEB2F
:1045F000F0A3EAF0A3E9F02425F9E43AFA900C7B61
:104600007401F0A3740CF0A37476F0125059EF60AB
:1046100008E4900B52F0A3F022784D768F08769143
:10462000E47821F60876650876C3900C71E0C4330F
:104630003354C0FF08F6A3E0FE1313543F4FF6EEC9
:10464000C4333354C0FF08F6A3E0FBA3E0FAA3E0B1
:10465000F912015EFE900C76E06EFE1313543F4F8C
:10466000F6EEC4333354C0FF08F6E92401F9E43A06
:10467000FA12015EFE900C77E06EFE1313543F4F6A
:10468000F6AF06EFC4333354C0FF08F6900C6EE06B
:10469000FBA3E0FAA3E02425F9E43AFA12015EFE56
:1046A0001313543F4FF6EEC4333354C0FF08F69053
:1046B0000C6EE0FBA3E0FAA3E02426F9E43AFA1238
:1046C000015EFE1313543F4FF6EEC4333354C0085B
:1046D000F67D367F0D1274C67F8F1275FCE4900B49
:1046E00052F0A3F0900C83741DF0A3E4F0A37400C7
:1046F000F0A37421F0A37409F07B007A00794E7D59
:1047000001126CE4900C6E125AE322900C6AEFF0E6
:104710007F05127340900C6C12733C900C6BEFF0A1
:10472000543CF030E21A900C6AE0244BF0E0D36481
:104730008094854037E024FBF0A3E04401F0802C16
:10474000900C6AE02447F0E0C3648094884009E05C
:1047500024F8F0A3E04401F0900C6AE0D364809464
:10476000765009E0240AF0A3E04402F0900C6AE0DD
:10477000FDD3648094804031900C6CE0547FF0ED68
:1047800075F00312013C900C6DF0D3940340037458
:1047900003F0900C6AE0FF900C6DE075F003A4FE4E
:1047A000C3EF9E900C6AF0803B900C6CE04480F06C
:1047B000900C6AE0FF3395E0FEC374029FFFE49E15
:1047C000FE7C007D031201BD900C6DEFF0D39403CD
:1047D00040037403F0900C6DE075F003A4FF900C9F
:1047E0006AE02FF0900C6BE0FF900C6DE0C4333367
:1047F00054C0FEEF4E900C6BF0A3E0FD7F051274E9
:10480000C6900C6BE0FD7F0A1274C6900C6AE0FF44
:1048100022E4900C5EF0900E27E0900C5DF01237D1
:104820005F900C5EEFF0E060030248CE12686D907E
:104830000B11E07002A3E07009900C5E7409F002A5
:1048400048CE900E2AE0700CA3E07008A3E070043C
:10485000A3E06024900C627401F0A3740EF0A374C2
:104860002AF0900B44E0FBA3E0FAA3E0F9123A78B7
:10487000900C5EEFF0E07056900E2EE0900C5BF026
:10488000FE900E29E0FF900C637401F0A3740EF00B
:10489000A3742FF0A3EEF0900E28E0900C67F0A325
:1048A0007401F0A3740CF0A3745EF0900B44E0FB71
:1048B000A3E0FAA3E0F9125417900C5CEFF0900C0F
:1048C0005BE06F6009900C5EE0700374FFF0E4FF42
:1048D0001273D9900D757436F0A37404F0900C5EC9
:1048E000E0900D77F0900C5CE0900D78F0900E7CED
:1048F000E0FBA3E0FAA3E02401F9E43AFA12015E36
:10490000900E7BF0A37401F0A3740DF0A37475F006
:104910007F36024DEA900C5CEBF0A3EAF0A3E9F0DD
:104920002425F9E43AFA900C7B7401F0A3740CF09E
:10493000A37462F0125059EF6008E4900B52F0A398
:10494000F022784D768F087691E47821F60876800B
:104950000876E0087602900C5FE0FBA3E0FAA3E0A3
:10496000F912015EFF900C62E0FE6F08F6E9240187
:10497000F9E43AFA12015EFF900C63E0FD6F08F66D
:10498000900C5FE0FBA3E0FAA3E02402F9E43AFA1A
:1049900012015EFFEE6F08F6900C5FE0FBA3E0FAF9
:1049A000A3E02403F9E43AFA12015EFFED6F08F682
:1049B000900C5CE0FBA3E0FAA3E02425F9E43AFACA
:1049C00012015E08F6900C5CE0FBA3E0FAA3E02481
:1049D00026F9E43AFA12015E08F67D367F0D12746C
:1049E000C67F8F1275FCE4900B52F0A3F0900C83FD
:1049F000741DF0A3E4F0A37400F0A37421F0A37479
:104A00000AF07B007A00794E7D01126CE4900C5C18
:104A1000125AE322900C7FEBF0A3EAF0A3E9F0AC8A
:104A2000071254D1900C8EEFF0E4900C83F0EF332A
:104A300095E0FEEF25E0FFEE33FE748B2FF9740E48
:104A40003EFA7B01E4FD122D92900C8EE02FF09047
:104A50000C82E0900C84F0FD900C8E122D7B900C5B
:104A60008EE02FF0AF04900C85EFF0FD900C8E12CD
:104A70002D7B900C8EE02FF0A37403F0900C8FE050
:104A8000FFC36480948B505B900C7FE0FBA3E475C4
:104A9000F001120209A9F0FA12015EFEEFFD339552
:104AA000E0FC74832DF582740C3CF583EEF0900CE1
:104AB0008EE0FF3395E0FEEF25E0FFEE33FE748BD2
:104AC0002FF9740E3EFA7B0174832DF582740C3C31
:104AD000F583E0FD122D92900C8EE02FF0A3E00400
:104AE000F080997B017A0C79837D0B7C00126058F1
:104AF000AD07AC06900C8E126DA2900C8EE02FF0DC
:104B00007B017A0E798BE0FD3395E0FC027497907F
:104B10000C8AEBF0A3EAF0A3E9F0A3EDF0E4FFA325
:104B2000E0FBA3E0FAA3E0F912015EFE900C8AE03C
:104B3000FBA3E0FAA3E02402F9E43AFAEE120199A9
:104B4000900C8EE0FBA3E0FAA3E02401F9E43AFA2A
:104B500012015EFE900C8AE0FBA3E0FAA3E02403BE
:104B6000F9E43AFAEE120199900C8DE0FEEFC39E43
:104B70005032900C91E0FBA3E0FAA3E02FF9E43A65
:104B8000FA12015EFE900C8AE0FBA3E0FAA3E02497
:104B900004F9E43AFAEF7C0029F9EC3AFAEE120152
:104BA000990F80C4900C8DE0FF900C8AE0FBA3E08D
:104BB000FAA3E02424F9E43AFAEF120199900C9454
:104BC000E0FBA3E0FAA3E0F912015EFF900C8AE09B
:104BD000FBA3E0FAA3E02425F9E43AFAEF120199E5
:104BE000900C94E0FBA3E0FAA3E02401F9E43AFA84
:104BF00012015EFF900C8AE0FBA3E0FAA3E02426FA
:104C0000F9E43AFAEF020199900C5CEBF0A3EAF0B8
:104C1000A3E9F02425F9E43AFA900C7B7401F0A39F
:104C2000740CF0A37462F0125059EF6008E4900B1A
:104C300052F0A3F022784D768F087691E47821F631
:104C40000876700876E008760708F6900C5FE0FBBF
:104C5000A3E0FAA3E0F912015EFF900C62E06F0896
:104C6000F6E92401F9E43AFA12015EFF900C63E0E0
:104C70006F08F6900C5CE0FBA3E0FAA3E02425F9B2
:104C8000E43AFA12015E08F6900C5CE0FBA3E0FA4D
:104C9000A3E02426F9E43AFA12015E08F67D367F95
:104CA0000D1274C67F8F1275FCE4900B52F0A3F0C6
:104CB000900C83741DF0A3E4F0A37400F0A374219E
:104CC000F0A37409F07B007A00794E7D01126CE448
:104CD000900C5CE0FBA3E0FAA3E02425F9E43AFAA7
:104CE000C002C001A3E0F9A3E0FAA3E0900C67C9F9
:104CF000F0A3EAF0A3E9F0D001D00212511D22E4A2
:104D0000900C8DF0900C8CF0900C8CE0FFC39419FB
:104D10005059EF64126013EF6414600EEF64156075
:104D200009EF64166004EFB41722900C8DE0FF04C5
:104D3000F0EF75F003A424A7F9740C35F0FA7B01A9
:104D4000900C8CE0FF7D031270C38017900C8CE0F8
:104D5000FF127340900C8CE0248EF582E4340CF545
:104D600083EFF0900C8CE004F0809DC2A17F017E67
:104D700000127641D2A17F017E00127641E4900CB0
:104D80008DF0900C8CF0900C8CE0FFC3941950596E
:104D9000EF64126013EF6414600EEF64156009EFA6
:104DA00064166004EFB41726900C8DE0FF04F0EF5A
:104DB00075F003A424A7F9740C35F0FA7B01900C6C
:104DC0008CE0FF900CBA7403F0126B038013900C0C
:104DD0008CE0FF248EF582E4340CF583E0FD127440
:104DE000C6900C8CE004F0809D22900C6AEFF0A33A
:104DF0007403F0A374E8F0900E7BE0FFA3E0FBA344
:104E0000E0FAA3E02401F9E43AFAEF120199900FD5
:104E10002BE064017031900F2BE0B40117900C6B04
:104E200074FFF5F01201F345F060097F647E001213
:104E3000784D80E2900C6BE07002A3E070097BFF7C
:104E40007A7679EF121083E4900C6AF0A2AF9201A7
:104E5000C2AFE59620E7FB75960E759701E59620A3
:104E6000E7FB759691E59620E7FBAF97900F2BE057
:104E7000FEB4030DE59620E7FB759611759710803B
:104E800046EE7043900F2B04F0EF30E50BE59620D3
:104E9000E7FB759611759740EF30E20BE59620E73A
:104EA000FB759611E4F597900E7BE0FD7C00A3E086
:104EB000FBA3E0FAA3E0F97F21126DFAE59620E763
:104EC000FB759611759701A20192AF22900C5C744C
:104ED000FFF0E4900C5BF0900C5BE0FFFDD3900BD7
:104EE00012E09D900B11E09400405FEF75F028A454
:104EF0002415F9740135F0FA7B0178287C0E7D01C8
:104F00007E007F081205A8EF703812375F900C5CA6
:104F1000EFF07029900E30E0FD900C827401F0A348
:104F2000740DF0A37479F0900E31E0900C85F07B55
:104F3000017A0E7928124119900C5CEFF0E4FF120F
:104F400073D9900C5BE004F0808D900D757450F077
:104F5000A37440F0900C5CE0FF3395E0FE7CFF7D95
:104F6000FF1201AB900D77EFF0900E31E0900D78CD
:104F7000F07B017A0D7975900E7CEBF0A3EAF0A33B
:104F8000E9F02401F9E43AFA12015E900E7BF07F19
:104F900050024DEA900C5FEBF0A3EAF0A3E9F07841
:104FA0004D768F087691E47821F60876590876C513
:104FB000A3E0FBA3E0FAA3E0F912015E08F6E924FE
:104FC00001F9E43AFA12015E08F6900C5FE0FBA3E7
:104FD000E0FAA3E02425F9E43AFA12015EFFC45492
:104FE0000FFE900C62E0FBA3E0FAA3E02402F9E4D8
:104FF0003AFA12015E54F04E08F6900C5FE0FBA303
:10500000E0FAA3E02426F9E43AFA12015EFEC45461
:105010000FFDEFC454F04D08F6EEC454F008F67DD1
:10502000367F0D1274C67F8F1275FCE4900B52F020
:10503000A3F0900C83741DF0A3E4F0A37400F0A31C
:105040007421F0A37408F07B007A00794E7D011280
:105050006CE4900C5F125AE322900C7E7401F0789D
:105060004D768F087690E47821F60876300876C180
:1050700012015E08F6E92401F9E43AFA12015E0829
:10508000F6E4900B52F0A3F0FD7F1A1274C67D2057
:105090007F1B1274C67F8F1275FC900C83741DF0F9
:1050A000A3E4F0A37400F0A37421F0A37405F07BD3
:1050B000007A00794E7D01126CE47F807E001269D7
:1050C000B97F8F1275FC7F5F7E001269B9900B5318
:1050D000E030E629E0541E6008900C7E7401F080F8
:1050E00028E4900B52F0A3F0900C7BE0FBA3E0FAD5
:1050F000A3E0F91278E1E4900C7EF0800CE4900BD0
:1051000052F0A3F0900C7E04F0E4FD7F1B1274C6F5
:10511000E4900B52F0A3F0900C7EE0FF22900C6420
:10512000EBF0A3EAF0A3E9F0900C6A7404F07F803E
:105130007E001269B9E4900B52F0A3F07F8F1275D4
:10514000FC7D3F7F0D1274C67D147C007F527E0073
:1051500012666C900B53E030E677900C67E0FBA38F
:10516000E0FAA3E0F97F021278A77B017A0C796B51
:105170007F021278A77F8F1275FC900B53E030E30B
:1051800023900C67E0FBA3E0FAA3E0F912015E4470
:1051900080120199900C67E0FBA3E0FAA3E0F912FA
:1051A000015E8029900C64E0FBA3E0FAA3E0F91211
:1051B000015EFF900C6BE06F6012E92401F9E43AA4
:1051C000FA12015EFF900C6CE0B50705E4900C6AE2
:1051D000F0E4900B52F0A3F0900C6AE0FF22900CE8
:1051E0005C74FDF0E4900C5BF0900C5BE0FFFDD391
:1051F000900B12E09D900B11E09400405FEF75F072
:1052000028A42415F9740135F0FA7B0178287C0E66
:105210007D017E007F081205A8EF703812375F907D
:105220000C5CEFF07029900E30E0FD900C61740181
:10523000F0A3740EF0A37432F0900E31E0900C6481
:10524000F07B017A0E7928123114900C5CEFF0E4B7
:10525000FF1273D9900C5BE004F0808D900D757493
:1052600048F0A37403F0900C5CE0FF3395E0FE7C03
:10527000FF7DFF1201AB900D77EFF07B017A0D7986
:1052800075900E7CEBF0A3EAF0A3E9F02401F9E4B9
:105290003AFA12015E900E7BF07F48024DEA900FC1
:1052A00020E07010A3E0700C900F24E07006A3E0E3
:1052B0006402600312769C900F1EE0247F6013143A
:1052C000603224027072900F22E07017A3E0601524
:1052D0008066900F1AE0B4040A900F22E07004A3D5
:1052E000E060028053900F1B74FFF0A37480F0A362
:1052F00074BF8036900F1AE0B40406900F22E0606D
:10530000028035900F23E0B4812C900F2BE0900F9A
:105310001BB4030C74FFF0A37480F0A374BD800A67
:1053200074FFF0A37480F0A374BFF0900F28E4F032
:10533000A37402F08005800012769C900F2AE0642E
:10534000046018E59620E7FB759611759740900F5D
:105350002A7401F0E4900F26F0A3F022900C5BE495
:10536000F0A3F0A3F0900B54E0B40110900C5B7428
:10537000FFF0A37461F0A37482F08038900E28E0EF
:10538000146013047020900C5B74FFF0A37461F040
:10539000A37496F0801E900C5B74FFF0A37461F010
:1053A000A374B9F0800E900C5B74FFF0A37461F0ED
:1053B000A374DBF07F31900D77E4F0A3DFFC900D58
:1053C000757411F0900C5BE0FBA3E0FAA3E0F91216
:1053D000758EEF04900D76F0900CDC7401F0A374E0
:1053E0000DF0A37477F0900D76E024FE900CDFF0C2
:1053F000900C5BE0FBA3E0FAA3E0F9127190900E31
:105400007C7401F0A3740DF0A37475F0900E7B749E
:1054100031F07F11024DEA900C5FEFF0A3EBF0A3A7
:10542000EAF0A3E9F0E4900C6BF0A3F0900C66E0D6
:10543000FF900C6CE0C39F40030254CBE4A3F090B8
:105440000C6CE0FC900C5FE02C900C72F0EC75F0B2
:1054500002A4FF900C63E0FBA3E0FAA3E02FF9EABB
:1054600035F0FA900C73EBF0A3EAF0A3E9F0900C9E
:1054700067E0FD900C60E0FBA3E0FAA3E0F91245C1
:10548000E7900C6BEFF0900C6DE004F0E0C3940734
:10549000500C900C6BE0600612753FEF70A1900B02
:1054A0003BE06006900C6B740AF0900C6BE0FF60C0
:1054B00011900C68E0FBA3E0FAA3E0F9EF12019968
:1054C0008009900C6CE004F002542C900C6CE0FF0E
:1054D000227B017A0E798B900C94EBF0A3EAF0A377
:1054E000E9F0900C94E0FBA3E0FAA3E0F974551204
:1054F0000199900C94E0FBA3E0FAA3E02402F9E404
:105500003AFA7455120199900C94E0FBA3E0FAA3C7
:10551000E02404F9E43AFA7473120199900C94E0CF
:10552000FBA3E0FAA3E02406F9E43AFA740A1201B4
:1055300099900C94E0FBA3E0FAA3E02401F9E43A8B
:10554000FA7408120199900C94E0FBA3E0FAA3E02E
:105550002403F9E43AFA7408120199900C94E0FBE0
:10556000A3E0FAA3E02405F9E43AFA7408120199D9
:10557000900C94E0FBA3E0FAA3E02407F9E43AFAE4
:105580007404120199FF22900B47E0B40102E4F089
:10559000900E28E06006A3E0900B3CF0900E2AE00D
:1055A0006006A3E0900B3DF0900E2CE06006A3E0B7
:1055B000900B3EF0900E2EE06006A3E0900B3FF0C3
:1055C000900E30E06006A3E0900B43F0900E32E0C6
:1055D0006006A3E0FF12470B7E007F407D007B0149
:1055E0007A0D79751205CC900D75745AF0A374403C
:1055F000F0900B3CE0900D78F0900B3DE0900D7A30
:10560000F0900B3EE0900D7CF0900B3FE0900D7E13
:10561000F0900B43E0900D80F0126BBF900D82EF85
:10562000F0900E7B7440F0A37401F0A3740DF0A30E
:105630007475F07F5A024DEA900C5CEBF0A3EAF02F
:10564000A3E9F0784D768F087691E47821F6087614
:10565000430876E0087603ED60050876808004E470
:105660007825F6900C5CE0FBA3E0FAA3E02425F992
:10567000E43AFA12015EFF54FEC313782546F6EFB2
:105680005401C43333335480FF900C5CE0FBA3E03F
:10569000FAA3E02426F9E43AFA12015EFE54FEC3AE
:1056A000134F08F6EE5401C4333333548008F67DAB
:1056B000367F0D1274C67F8F1275FCE4900B52F08A
:1056C000A3F0900C83741DF0A3E4F0A37400F0A386
:1056D0007421F0A37407F07B007A00794E7D0112EB
:1056E0006CE4900C5C125AE322900F58EBF0A3EAA2
:1056F000F0A3E9F0900F58E0FBA3E0FAA3E0240246
:10570000F9E43AFA12015E900CDCF0900F58A3E035
:10571000FAA3E02403F9E43AFA12015E900CDDF0FA
:105720007BFF7A5D79601210837BFF7A5D7974125A
:105730001083E4900F5BF0A3F0900F58E0FBA3E020
:10574000FAA3E02424F9E43AFA12015EFF900F5B19
:10575000E0FCA3E0FDC39FEC94005034900F58A3ED
:10576000E0FAA3E02404F9E43AFAE92DF9EA3CFA74
:1057700012015E900CDCF07BFF7A5D797F12108362
:10578000900F5CE004F070B1900F5BE004F080A932
:105790007BFF7A5D7985021083C0E0C0F0C083C0D2
:1057A00082C0D075D000C000C001C002C003C004D8
:1057B000C005C006C007E59620E7FB759686E5960E
:1057C00020E7FB900CD5E597F0E59620E7FB759672
:1057D00082E59620E7FB900CD6E597F0E59620E76A
:1057E000FB759684E59620E7FB900CD7E597F09043
:1057F0000CD5E030E1031277F3900CD5E030E203F2
:1058000012767F900CD6E030E0031214BD900CD6D7
:10581000E030E1031278AE900CD7E030E10312687B
:10582000DF900CD5E030E003127802D007D006D02C
:1058300005D004D003D002D001D000D0D0D082D087
:1058400083D0F0D0E032E4900C5BF0126B5B123747
:105850005F900C5BEFF0E4900B11F0A3F0EF70376A
:105860007B01900C6504F0A3740EF0A37429F090F2
:105870000E28E0900C68F0E4A3F0A374FFF0A3748A
:1058800075F0A3743FF07A0179117D0112230E9017
:105890000B11EEF0A3EFF0E4FF1273D9900B11E0BF
:1058A0007002A3E0900B4460127401F0A37401F045
:1058B000A37411F0E4900C5BF0800CE4F0A3F0A36F
:1058C000F0900C5B7409F0900D757434F0A37403C0
:1058D000F0900C5BE0900D77F0900E7B7403F0A3DA
:1058E0007401F0A3740DF0A37475F07F34024DEAD7
:1058F000C0E0C0F0C083C082C0D075D000C000C07E
:1059000001C002C003C004C005C006C0071278C6AB
:10591000900B51EFF01278C6AC07900B4EE4F0906C
:105920000B51E0FE4F543F900D22F0EE54C0FF604B
:1059300009E0FEECF45FFFEE4FF0900D22E0900BDB
:1059400051F030E5231278C0900B4EEFF0541FC396
:1059500094124004E04480F0900B4EE0FF541FD3BB
:1059600094065004EF4440F0900B4EE0FE900D2260
:10597000E0FDEDFF900B52E04EF0A3E04FF0D007BA
:10598000D006D005D004D003D002D001D000D0D0B2
:10599000D082D083D0F0D0E032900C5CEBF0A3EA60
:1059A000F0A3E9F02425F9E43AFA900C7B7401F0B5
:1059B000A3740CF0A3745FF0125059EF6008E490E8
:1059C0000B52F0A3F022784D768F087691E478217F
:1059D000F60876400876E0087601900C5CE0FBA3C0
:1059E000E0FAA3E02425F9E43AFA12015E08F69001
:1059F0000C5CE0FBA3E0FAA3E02426F9E43AFA12F7
:105A0000015E08F67D367F0D1274C67F8F1275FC1D
:105A1000E4900B52F0A3F0900C83741DF0A3E4F01B
:105A2000A37400F0A37421F0A37406F07B007A0045
:105A3000794E7D01126CE4900C5C125AE322900CBA
:105A40005CEBF0A3EAF0A3E9F02425F9E43AFA903C
:105A50000C7B7401F0A3740CF0A3745FF012505926
:105A6000EF6008E4900B52F0A3F022784D768F0897
:105A70007691E47821F60876400876E0087605907D
:105A80000C5CE0FBA3E0FAA3E02425F9E43AFA1267
:105A9000015E08F6900C5CE0FBA3E0FAA3E024268C
:105AA000F9E43AFA12015E08F67D367F0D1274C6EB
:105AB0007F8F1275FCE4900B52F0A3F0900C83746E
:105AC0001DF0A3E4F0A37400F0A37421F0A3740606
:105AD000F07B007A00794E7D01126CE4900C5C1230
:105AE0005AE322E0FBA3E0FAA3E02425F9E43AFA22
:105AF000900C78EBF0A3EAF0A3E9F0A37404F07F34
:105B0000807E001269B9E4900B52F0A3F07F8F12EF
:105B100075FC7D3F7F0D1274C67D147C007F527E24
:105B20000012666C900B53E030E64D7B017A0C79E5
:105B30007C7F021278A77F8F1275FC900B53E030A8
:105B4000E309900C7CE04480F08029900C78E0FB25
:105B5000A3E0FAA3E0F912015EFF900C7CE06F6015
:105B600012E92401F9E43AFA12015EFF900C7DE09B
:105B7000B50705E4900C7BF0E4900B52F0A3F09095
:105B80000C7BE0FF2225686878202568687820254E
:105B900068687820256868780A00454E2070696E2C
:105BA000206661696C65640A0043616E6E6F7420E3
:105BB00072756E206F6E204153333939300A0043BD
:105BC000616E6E6F742072756E206F6E204153335C
:105BD0003939310A00556E6B6E6F776E20636869D4
:105BE0007020256868780A00494E5456434F5F6C10
:105BF000776D0A005449204F2054202578202578BD
:105C00000A005449204F2025782025780A000A727E
:105C1000656720256868782020200025686878203E
:105C20000025686878007B017A0C79677D08900C04
:105C300094EBF0A3EAF0A3E9F0A3EDF0E4900C9A62
:105C4000F0900B52E0FFA3E0900C98CFF0A3EFF0A0
:105C5000E4900B52F0A3F07D067F011274C67D0321
:105C6000E4FF1274C6900C98E0FEA3E0FF30E1065A
:105C7000A374FBF08044EF30E408900C9A74FFF0BA
:105C80008038EF30E62E7F1C127340EF541FFE90D9
:105C90000C97E0FFB50615900C94E0FBA3E0FAA387
:105CA000E0F91278A7E4900C9AF0800E900C9A74A8
:105CB000FEF08006900C9A74FDF07F8F1275FC90B8
:105CC0000C9AE0FF22E4900F54F0E4900F55F0A3FB
:105CD000F0A3F0900F53F0900C65E4F0A3F0A3F064
:105CE000A3F0900F54E0900C69F0A374FFF0A3743C
:105CF00078F0A374F9F07B017A0179117D101223F9
:105D00000EEFFD900F57E02DF0900F56E03400F0AD
:105D1000900F55E0FEEFD39E4002EFF0900F53E05E
:105D200004F0E0C394FF40AF7BFF7A64794E900F9C
:105D300054E0900CDCF0900F56E0FFA3E0900CDDF7
:105D4000CFF0A3EFF0900F55E0900CDFF01210832E
:105D5000900F54E004F0E0C3940F5003025CCA2299
:105D60005072696E74205043202568687820256839
:105D700068780A005072696E7420455043200025EF
:105D800068687820000A0054414720256868783AFE
:105D90000A00524E31363A20256868782025686816
:105DA000780A004E756D626572206F6620726561BB
:105DB000642062797465733A2025640A0050433A7E
:105DC00020256868782025686878004550433A2087
:105DD000004550434C454E20286279746573293A3A
:105DE00020256868640A0048414E444C453A202505
:105DF00068687820256868780A00ED603575A5FF29
:105E0000900D2EE06010C2A8C2A0E4F590D2A0755B
:105E100090800000C2A0AF051DEF601612015EF574
:105E20009000D2A0000000C2A0740129F9E43AFA5F
:105E300080E4900D2CE06034E4F5A57590FF900DA2
:105E40002CE0FF14F0EF60247590FFD2A000900DBD
:105E500029E0FBA3E0FAA3E0F9E590120199C2A0C2
:105E6000900D2AE475F0011201F380D275A5FF9020
:105E70000D2DE0FFB4020DC2A0E4F59000759080F6
:105E80000000F590EFB4010B75908000D2A0E4F50E
:105E900090C2A022900C5BEFF0D3940F4003748962
:105EA000F0900C5BE0242DF582E4340FF583E09054
:105EB0000C5DF0E0C4135407900C5CF0900C5CE0B7
:105EC000FFD39400404DC2A2EF14FF74017E00A8DE
:105ED00007088005C333CE33CED8F9FF900C5DE0C0
:105EE000FDEF5D7BFF600D7A6479791210837FC2CC
:105EF0007E01800B7A64797B1210837F967E00127C
:105F00007641D2A27F967E00127641900C5CE0141E
:105F1000F080A97BFF7A64797D900C5BE0900CDCCB
:105F2000F01210837FC27E01027641900D75741DC0
:105F3000F0900E28E0FF64126013EF6414600EEF1F
:105F400064156009EF64166004EFB417287B017ACA
:105F50000C795B7D031270C3900CDC7401F0A374A8
:105F60000DF0A37477F0A37403F07B017A0C795BD6
:105F7000127190802E900E28E0FF127340900C5BFF
:105F8000EFF0900CDC7401F0A3740DF0A37477F0C3
:105F9000A37401F0FB7A0C795B127190E4900D7898
:105FA000F0A3F0900D75741DF0A37406F0900E7BB5
:105FB000F0A37401F0A3740DF0A37475F07F1D02BB
:105FC0004DEA900C5C7402F0900D757458F0E490FA
:105FD0000C5BF0900C5BE0FFC3941F505AEF64120F
:105FE0006013EF6414600EEF64156009EF641660CF
:105FF00004EFB4171D900C5CE07C002475F9EC34C0
:106000000DFA7B017D031270C3900C5CE02403F059
:10601000801D900C5BE0FF127340900C5CE02475D7
:10602000F582E4340DF583EFF0900C5CE004F09021
:106030000C5BE004F0809C900C5CE02402900D76F8
:10604000F0900E7B7440F0A37401F0A3740DF0A3E4
:106050007475F07F58024DEA900C94EBF0A3EAF0CF
:10606000A3E9F0A3ECF0A3EDF074FF900C9BF0A378
:10607000F0E4900C99F0A3F0900C97E0FEA3E0FF01
:10608000C3900C9AE09FEE6480F8900C99E06480D5
:10609000985051900C94E0FBA3E475F001120209B2
:1060A000A9F0FA12015EFD900C9BE0FAA3E0FBEA76
:1060B000FFEF6D25E0FFE433FE74BD2FF582747EA3
:1060C0003EF583EBFEE4936EFF740193900C9BCF3F
:1060D000F0A3EFF0900C9AE004F0709C900C99E023
:1060E00004F08094900C9BE0FEA3E0FF22E4900F6C
:1060F00062F0900F62E0FFC3941F40030261817B56
:10610000FF7A5C790E900CDCEFF0121083900F6236
:10611000E0FF64126014EF6414600FEF6415600A0E
:10612000EF64166005EF641770387A0F79631270A8
:10613000BF7BFF7A5C791B900F65E0900CDCF0125E
:1061400010837BFF7A5C791B900F64E0900CDCF08D
:106150001210837BFF7A5C791B900F63E0900CDC5C
:106160008012900F62E0FF1273407BFF7A5C79210E
:10617000900CDCEFF0121083900F62E004F00260EC
:10618000F22263617574696F6E2077726F6E67209B
:10619000636869700A00415333393932204D696EA2
:1061A0006920526561646572204669726D7761721B
:1061B0006520312E352E310A0041533339393220D2
:1061C000524F4745522052656164657220486172A2
:1061D000647761726520312E330A0057726F6E67E3
:1061E0002076657273696F6E2074797065207365AF
:1061F0006E64004B494C4C205461670A006E6F205E
:106200006E65656420746F206163636573732054E9
:1062100061670A00900F6AEBF0A3EAF0A3E9F0745B
:1062200030120199900F6AE0FBA3E0FAA3E0240189
:10623000F9E43AFA7478120199EF7804A2E713D8D6
:10624000FB540FFED394095005EE2430800574F6FC
:106250002E2441FD900F6AE0FBA3E0FAA3E02402A4
:10626000F9E43AFAED120199EF540FFED394095074
:1062700005EE2430800574F62E2441FF900F6AE06D
:10628000FBA3E0FAA3E02403F9E43AFAEF12019940
:10629000900F6AE0FBA3E0FAA3E02404F9E43AFAE1
:1062A000E40201997BFF7A6179F312108312375F60
:1062B000900C5BEFF0703E12686D900B11E0700275
:1062C000A3E07008900C5B7409F08029900C5F7457
:1062D00001F0A3740EF0A37428F0900E2CE0900C43
:1062E00062F0900B44E0FBA3E0FAA3E0F91244C390
:1062F000900C5BEFF0E4FF1273D9900D75743EF0D3
:10630000A37404F0900C5BE0900D77F0900E7CE0AD
:10631000FBA3E0FAA3E02401F9E43AFA12015E904B
:106320000E7BF0A37401F0A3740DF0A37475F07FDD
:106330003E024DEA787FE4F6D8FD75815075D900AC
:1063400002637E020BBBE493A3F8E493A34003F63D
:106350008001F208DFF48029E493A3F85407240CA9
:10636000C8C333C4540F4420C8834004F45680018A
:1063700046F6DFE4800B01020408102040809027DD
:10638000E9E47E019360BCA3FF543F30E509541F4C
:10639000FEE493A360010ECF54C025E060A840B88E
:1063A000E493A3FAE493A3F8E493A3C8C582C8CA0C
:1063B000C583CAF0A3C8C582C8CAC583CADFE9DEDF
:1063C000E780BE900F1AE064047061900F1EE0FF3A
:1063D000605A64016056900F20E07050900F22E0E8
:1063E000704A900F24E07044A3E06002803E900F5A
:1063F0001EE064027036900F21E07030900F23E0B1
:10640000FF64816005EF64027022EFB48121E5969C
:1064100020E7FB75960E759701E59620E7FB7596CC
:1064200011759710900F2B7403F0800312769CE582
:106430009620E7FB75960EE4F597900F2AE064042A
:10644000600BE59620E7FB75961175974822666FFD
:10645000756E64207769746820706F77536C6F7401
:106460003D2568687820257820746167732C206D3D
:10647000617820256868780A002D002E00202568A4
:1064800068780A0048656C6C6F20726F67657220CF
:10649000554846205246494420576F726C640A00A2
:1064A0006C776D5F617333393978496E69746961EE
:1064B0006C697A6528292072657475726E6564202E
:1064C00025780A007573625F696E697420636F6D69
:1064D000706C657465210A00900F1AE064026025F3
:1064E000900F1EE0701F900F22E07019A3E070154E
:1064F000A3E07011A3E0700D900F20E07007A3E0FF
:10650000D39401400512769C8044900F21E0D394EF
:10651000004031900F1A7404F0E4900F2BF0E596D0
:1065200020E7FB75960E759701E59620E7FB7596BB
:1065300012759704E59620E7FB75960EE4F5971221
:1065400078AE800A900F1A7403F0900F2BF0900F22
:106550002AE06404600BE59620E7FB7596117597B9
:106560004822900F1AE06404705B900F1EE0FF60F9
:106570005464016050900F20E0704A900F22E07048
:1065800044900F24E0703EA3E060028038900F1E1C
:10659000E064027030900F21E0702A900F23E0FF3A
:1065A00064817021EFB48120E59620E7FB75960E9B
:1065B000759701E59620E7FB759611759740E49075
:1065C0000F2BF0800312769CE59620E7FB75960E64
:1065D000E4F597900F2AE06404600BE59620E7FB52
:1065E00075961175974822900E28E0FF900C5BF08D
:1065F00064126014E0FE6414600EEE64156009EE2F
:1066000064166004EEB417117B017A0E7929900CA0
:10661000BA7403F0126B03801E900C5BE0C394808D
:10662000500D900E28E0FFA3E0FD1274C680089084
:106630000C5BE0FF1275FC900D75741BF0A37403E6
:10664000F0E4A3F0900E7CE0FBA3E0FAA3E02401C9
:10665000F9E43AFA12015E900E7BF0A37401F0A304
:10666000740DF0A37475F07F1B024DEA900C7EEE62
:10667000F0A3EFF0A3ECF0A3EDF0900C7EE0FEA30E
:10668000E0FF900B52E05EFEA3E05F4E7026900CA0
:1066900080E07002A3E0601CE59130E7DD7FE87EDA
:1066A000031275B3900C81E024FFF0900C80E0346D
:1066B000FFF080C6900C80E07002A3E07032124CB4
:1066C000FF7BFF7A5B79F4900B52E0FFA3E0900C24
:1066D000DCCFF0A3EFF0900C7EE0FFA3E0900CDEA7
:1066E000CFF0A3EFF0121083900B52E4F0A304F06C
:1066F00022900F1EE06480701C900F20E07016A3A3
:10670000E07012A3E0700EA3E0700AA3E07006A38D
:10671000E06401600512769C8038900F1AE0FFB4A7
:106720000416900F1B74FFF0A37480F0A374BDF0E7
:10673000900F28E4F0A304F0EFB40316900F1B743D
:10674000FFF0A37480F0A374BFF0900F28E4F0A3CF
:1067500004F0900F2AE064046018E59620E7FB75CA
:106760009611759740900F2A7401F0E4900F26F06F
:10677000A3F022C0E0C083C082C0D075D000C000AA
:10678000C001C002C003C006C0077812E66051C253
:10679000CF08860308E6FA08E62401F9E43AFA7419
:1067A000FF120177FF7813860308E6FA08E6F9126C
:1067B000015EFEA807088002C313D8FCFF78138689
:1067C0000308E6FA08E62401F9E43AFA12015E70D9
:1067D0000B740226F618E436F6781216EF1392932D
:1067E000D007D006D003D002D001D000D0D0D082C4
:1067F000D083D0E032900F5DEBF0A3EAF0A3E9F094
:106800001278CC900F61EFF0900F607433F0C2A853
:10681000900D29E4F0A3F0A3F0A3F0A3F0A304F0FB
:10682000FB7A0F7960FD125DFA900D29E4F0A3F078
:10683000A3F0A3F0A3F0A3F07B017A0F79617D01AF
:10684000125DFA900F5DE0FBA3E0FAA3E02401F9EA
:10685000E43AFA900D29E4F0A3F0A3F0A3F0A374B6
:1068600002F0E4A3F07DFB125DFAD2A822900B4463
:10687000A3E0FAA3E04A7003FEFF22900B44E0FB82
:10688000A3E0FAA3E02404F9E43AFA900C65EBF0F3
:10689000A3EAF0A3E9F0900B44A3E0FAA3E02424D8
:1068A000F9E43AFA12015E900C68F0E4A3F0A374E4
:1068B000FFF0A37475F0A3743FF07B017A0179397E
:1068C0007D0112230E900B11EEF0A3EFF04E600E3F
:1068D000900B447401F0A37401F0A37439F022E426
:1068E000900CD8F0E59620E7FB75960E759701E5BC
:1068F0009620E7FB759694E59620E7FBAF97900FFF
:106900002BE0B4030CE59620E7FB759614759720F1
:1069100022EF30E60BE59620E7FB7596147597801D
:1069200012002E900E66E0FD7C00A37F21126C8485
:10693000900E67E0FBA3E0FAA3E0F912015EFF12FC
:106940006D42E59620E7FB759614E4F59722900CCE
:1069500076EFF07F8F1275FC784D768F087698E48D
:106960007821F6900EF2E03333335418FF900EF591
:10697000E0C43354204FFF900EF4E025E025E054AE
:10698000044FF6900C76E025E0541EFF900EF3E0E5
:10699000FEC4333354C04F08F6900C83741FF0A329
:1069A000E4F0A37400F0A37421F0A37402F07B0060
:1069B0007A00794E7D01026CE4900C8AEEF0A3EF30
:1069C000F0E4FFFE900C8AE0FCA3E0FD900B52E0A7
:1069D0005CFCA3E05D4C7010C3EF94FDEE94FF509F
:1069E000070FBF00010E80DCD3EF94F0EE94FF4060
:1069F00032124CFF7BFF7A5C7902900B52E0FFA3CE
:106A0000E0900CDCCFF0A3EFF0900C8AE0FFA3E065
:106A1000900CDECFF0A3EFF0121083900B52E4F055
:106A2000A304F022900F1AE064047024900F1EE07B
:106A30006481701C900F20E07016A3E07012A3E038
:106A4000700EA3E0700AA3E07006A3E06401600585
:106A500012769C8016900F1B74FFF0A37480F0A335
:106A600074BFF0900F28E4F0A304F0900F2AE064C4
:106A7000046018E59620E7FB759611759740900F16
:106A80002A7401F0E4900F26F0A3F022900C7EEF20
:106A9000F0D2937F017E001276411254D1900C7F88
:106AA000EFF03395E0FEEF25E0FFEE33FE748B2F21
:106AB000F9740E3EFA7B01900C7EE0FD122D92904F
:106AC0000C7FE02FF07B017A0C797E7D017C001237
:106AD0006058AD07AC06900C7F126DA2900C7FE061
:106AE0002FF07B017A0E798BE0FD3395E0FC127478
:106AF00097D29322F07A0C796F7B01900CBA7403D1
:106B0000F07F14900CB6EFF0A3EBF0A3EAF0A3E94A
:106B1000F0900CB6E04420F0C2A8900D29E4F0A358
:106B2000F0A3F0A3F0A3F0A304F0FB7A0C79B6FD78
:106B3000125DFA900CBAE0FD900D29E4F0A3F0A3E9
:106B4000F0A3F0A37402F0E4A3F0900CB7E0FBA371
:106B5000E0FAA3E0F9125DFAD2A822900C61740168
:106B6000F0A37401F0A37411F0E4FFFEFD8046E48D
:106B7000FF7E0AFDFC900C5DE0F8A3E0F9A3E0FACB
:106B8000A3E0FBC31203865035900C61E0FBA3E445
:106B900075F001120209A9F0FAE4120199900C5D56
:106BA000E0FCA3E0FDA3E0FEA3E02401FFE43EFE41
:106BB000E43DFDE43CFC900C5D1203BD80B122E499
:106BC000900C5BF07F05127340900C5C12733CEFED
:106BD00030E211900C5BE024B5F0EF30E020E024CF
:106BE00005F0801A900C5BE024B9F0EF30E004E08F
:106BF0002408F0EF30E107900C5BE024F6F0EFC4DE
:106C00001313540375F003A4FF900C5CE0900C5B2D
:106C100030E706E0C39FF08003E02FF0900C5BE0CC
:106C2000FF22900C76EBF0A3EAF0A3E9F0E4A3F0E6
:106C3000A3F07FC0FE1269B97F5F7E001269B99030
:106C40000B53E020E022E0541E6008900C7A74FFA1
:106C5000F08026900C76E0FBA3E0FAA3E0F9121A8C
:106C6000DF900C7AEFF08011900C76E0FBA3E0FA55
:106C7000A3E0F9E4F5F012024A7F8F1275FC900C44
:106C80007AE0FF22E0FBA3E0FAA3E0F9900CD9EF51
:106C9000F0900CDCEBF0A3EAF0A3E9F0900CDAEC56
:106CA000F0A3EDF04C603C900CD9E0F5964396C013
:106CB000E4FFFED3900CDBE09F900CDAE09E4020D6
:106CC000E59620E7FB900CDCE0FBA3E0FAA3E02FC5
:106CD000F9EA3EFAE5971201990FBF00010E80D341
:106CE000E4F59622900C83E04420F0C2A8900D2990
:106CF000E4F0A3F0A3F0A3F0A3F0A304F0125DFA74
:106D0000900D29E4F0A3F0A3F0A3F0A3F0A3F07B8F
:106D1000017A0C79837D01125DFA900C87E0FD9079
:106D20000D29E4F0A3F0A3F0A3F0A37402F0E4A310
:106D3000F0900C84E0FBA3E0FAA3E0F9125DFAD234
:106D4000A822900E7AE0703204F0900CDCF0A3746C
:106D50000EF0A37426F0900E67E0FBA3E0FAA3E028
:106D60002401F9E43AFA12015E04900CDFF0900E6F
:106D700067A3E0FAA3E0F9027190900E67E0FBA32D
:106D8000E0FAA3E0F912015E900CDCF0900E26E030
:106D9000900CDDF07BFF7A75791612108322AD0717
:106DA000AC06E0FF3395E0FEEF25E0FFEE33FE7426
:106DB0008B2FF9740E3EFA7B01900C94EBF0A3EA52
:106DC000F0A3E9F0A3ECF0A3EDF0F4FFECF4FE90F7
:106DD0000C97F0A3EFF0EEFD122D92900C95E47558
:106DE000F0041201F3900C94E0FBA3E0FAA3E0F9A5
:106DF000A3A3E0FD122D927F0422900C6DEFF09082
:106E00000C70EBF0A3EAF0A3E9F0900C6EECF0A3A9
:106E1000EDF04C603BE59620E7FB900C6DE0F596BD
:106E2000E4FFFED3900C6FE09F900C6EE09E40203C
:106E3000900C70E0FBA3E0FAA3E02FF9EA3EFA120F
:106E4000015EF597E59620E7FB0FBF00010E80D3AA
:106E500022900CD9EFF0900CDCEBF0A3EAF0A3E960
:106E6000F0900CDAECF0A3EDF04C603BE59620E7F7
:106E7000FB900CD9E0F596E4FFFED3900CDBE09F8D
:106E8000900CDAE09E4020900CDCE0FBA3E0FAA33B
:106E9000E02FF9EA3EFA12015EF597E59620E7FB4E
:106EA0000FBF00010E80D322900F1EE0701D900FC7
:106EB00022E07017A3E07013A3E0700FA3E0700B43
:106EC000900F20E07005A3E030E70312769C900F4E
:106ED0002A7405F0900F21E0900F1A60057403F0FA
:106EE00080037402F0900F2AE06404600BE59620A2
:106EF000E7FB7596117597482274142FF582740D6F
:106F00003EF583E0FF900DC1E0600BE4F0900DC012
:106F1000F07811E670FB900DC0E024C2F582E434F5
:106F20000DF583EFF0900DC0E004F0E0FDC3946434
:106F30005004EFB40A0F7B017A0D79C212740C90E1
:106F40000DC17401F022900CD9EFF0E4A3F0900C85
:106F5000DAE0FFD394035039EF25E025E0247FF5F4
:106F600082E4340EF583E0FF900CD9E0FEEFB50625
:106F700018A3E025E025E02480F582E4340EF583B3
:106F8000A3E0FAA3E0F90203EF900CDAE004F0804A
:106F9000BD22C0E0C083C082C0D075D000C000C098
:106FA00001C002C003C299790CE7780B66700578BE
:106FB00011F68018780D860308E6FA08E6F9780CD1
:106FC000E60629F9E43AFA12015EF599D003D002F7
:106FD000D001D000D0D0D082D083D0E032E596204E
:106FE000E7FB759601759708E59620E7FB75960710
:106FF000759707E59620E7FB759609759707E5965F
:1070000020E7FB75960B75970775D7E0E59620E7A7
:10701000FB75960F75978043E602D2AFE59620E7A1
:10702000FB75960175970122900F21E0FF126F46C4
:10703000900E7CE0F9A3E0FAA3E0900F1BC9F0A347
:10704000EAF0A3E9F0900E7BE0FF900F28E4F0A3B4
:10705000EFF0900F2AE064046018E59620E7FB75D6
:107060009611759740900F2A7401F0E4900F26F066
:10707000A3F02212002E900E67E0F9A3E0FAA3E03D
:10708000900F1BC9F0A3EAF0A3E9F0900F24E0FFF2
:10709000A3E0900F28CFF0A3EFF0900F2AE0640454
:1070A0006018E59620E7FB759611759740900F2ABA
:1070B0007402F0E4900F26F0A3F0227A0C796F7B33
:1070C000017D03900CB6EFF0A3EBF0A3EAF0A3E987
:1070D000F0C2A8900CB6E04460F0A3E0F9A3E0FA97
:1070E000A3E0900D29C9F0A3EAF0A3E9F0A3EDF025
:1070F000A37402F0A314F0FB7A0C79B6FD125DFACA
:10710000D2A8227F0A127340900C94EFF07D227F68
:10711000011274C6900C94E0FD7F0A1274C6E4FF5D
:107120001273727F8F1275FC7D507F1B1274C67FA5
:10713000971275FC7D43E4FF12761FC292D2937FB3
:10714000017E00127641C2A80278F5900E28E00474
:10715000600E147017D28243C701C2B0E4FF8009E9
:10716000C28253C7FED2B07F011273D9900D7574DD
:1071700019F0A37403F0E4A3F0900E7B7403F0A362
:107180007401F0A3740DF0A37475F07F19024DEA39
:10719000900CD9EBF0A3EAF0A3E9F0E4FF900CDF48
:1071A000E0FEEFC39E5029900CD9E0FBA3E0FAA3C8
:1071B000E02FF9E43AFA12015EFE900CDCE0FBA34A
:1071C000E0FAA3E02FF9E43AFAEE1201990F80CD2C
:1071D00022900C5DEFF0900B47E0FE6F6031EE24E3
:1071E000FE600804700812791E8003127914900C56
:1071F0005DE024FE600E04700E7B017A0B793C1278
:107200007917800312789F900C5DE0900B47F02275
:10721000D2937F067E00127641900C7574AAF0908E
:107220000C77F0900C79740AF0900C767408F0905A
:107230000C78F0900C7A7404F07B017A0C79757DEF
:10724000037C00127497D2937F017E00027641E4A2
:10725000780AF67811F6780BF608F6900DC1F090E2
:107260000DC0F0C29FD29D758840758920438E085D
:10727000758D30D28E43A41075E10175B283D2BCF6
:1072800075A890D2ACD2AF43E24022900F1EE064CA
:1072900001701C900F24E07016A3E07012900F2074
:1072A000E0700CA3E07008A3E07004A3E060031298
:1072B000769C900F2AE06404600BE59620E7FB754E
:1072C000961175974822900E27E0B40433900D75FF
:1072D0007456F0A37403F07B017A0D7975900E7CDF
:1072E000EBF0A3EAF0A3E9F02401F9E43AFA120181
:1072F0005E900E7BF0900D7774FFF07F56124DEA92
:107300002274FF900C5BF0A3F0EE3395E0FDFCE4FB
:107310007B30FAF9F8120269C374FF9F900C5CF09D
:1073200074FF9E900C5BF0E4F5C8438E30E0FEA342
:10733000E0FDF5CA8DCCEEF5CBF5CD22EFF07F0A5E
:10734000900D23EFF0C2A8E04440F0900D297401A5
:10735000F0A3740DF0A37424F0A37401F0A3F0A3C0
:10736000F0FB7A0D7923FD125DFAD2A8900D24E08E
:10737000FF22900C95EFF070077D407F091274C6D4
:10738000900C95E0B406077D807F091274C67F03D8
:10739000127340EF540FFF900C95E0FEC454F04F71
:1073A000FD7F030274C61278B4EF602C900E26E0C5
:1073B00075F003A4241FF582E5F03479F583E474B5
:1073C0000193FA740293F91203EF900B40E07003FB
:1073D0001278BAE4900B40F022900C6AEFF0E4FFD0
:1073E000127340900C6AE06008EF4401FFC2828093
:1073F00006EF54FEFFD282AD07E4FF1274C6900C74
:107400006AE060077F027E0012764122E4900D213F
:10741000F07811E670FB78117601780DA60308A6C6
:107420000208A601780C7601AF0518A607780D862C
:107430000308E6FA08E6F912015EF59922A2AF9276
:1074400000C2AF75FF8075EF028E088F0975B7A572
:1074500075B7F1438F0175FF8075EF02850982854D
:107460000883EDF0538FFEA20092AF22900D757449
:1074700005F0900D73E0900D76F0900D74E0900D96
:1074800077F0900E7C7401F0A3740DF0A37475F086
:10749000900E7B7403F0227813A60308A60208A6B8
:1074A00001E408F6AF057812A60775C804AFA87501
:1074B000A820D2AF7812E670FB30CFFD8FA8E4F59C
:1074C000C8227D02E4FF900CB6EFF0A3EDF0C2A855
:1074D000900D29E4F0A3F0A3F0A3F0A304F0A3F02F
:1074E000FB7A0C79B67D02125DFAD2A822900F6762
:1074F000EBF0A3EAF0A3E9F0900F67E0FBA3E0FA5A
:10750000A3E0F9127750AD07900F67E0FBA3E0FA14
:10751000A3E0F902740C757362206572726F7220B9
:107520002D207265706F72742025686878206C6FEA
:10753000737420616674657220256868780A00900B
:107540000B39E07002A3E070037F012212778DC334
:10755000900B3AE09F900B39E09E5009900B3B74E2
:1075600001F07F00227F01227F961275FC7F971227
:1075700075FC7FF47E0112784D7F0F127340900CE2
:107580007AEFF07F961275FC900C7AE0FF22900C57
:107590005EEBF0A3EAF0A3E9F0E4FF900C5EE0FB01
:1075A000A3E0FAA3E02FF9E43AFA12015E60030FB8
:1075B00080E9227C007D041203F5C374FF9FFF74F1
:1075C000FF9EFC538EBFE4F591EFFBF592ECF59333
:1075D0008B94F59543910422438E045388EF53D83E
:1075E000BFE58954F04401F589E4F58AF58C75D935
:1075F0000475D840F5F9F5FA43881022900C9BEFFA
:10760000F0C2A8900D29E4F0A3F0A3F0A3F0A30426
:10761000F0A3F0FB7A0C799BFD125DFAD2A82290C0
:107620000C95EFF0A3EDF0900D29E4F0A3F0A3F09A
:10763000A3F0A3F0A304F0FB7A0C79957D02025D20
:10764000FA900CB6EEF0A3EFF0900CB674FFF5F0E4
:1076500012020945F060097FE87E0312784D80E947
:107660002243B203E4F5B943B9801277E443B9C0C9
:107670001277E4E5B930E5FB75B69075A903229061
:107680000F1A7402F0E59620E7FB759601759701D5
:10769000E4900F2AF0A37403F0A3F022E59620E70C
:1076A000FB75960EE4F597E59620E7FB7596117548
:1076B0009720900F2A7404F0227F397E00E4FDFCAD
:1076C000C3ED9FEE6480F8EC64809850070DBD0018
:1076D000010C80EC2275F003EFA4241FF582E5F085
:1076E0003479F583740193FA740293F90203EF0A73
:1076F0000A53656E645061636B65742074696D65CF
:1077000064206F75740A0A00900E67E0FBA3E0FA2C
:10771000A3E02401F9E43AFA12015E900DBEF022D2
:10772000123E8E7F32124DEA900E287402F0900DB8
:1077300077E06003B401E9221229D67F32124DEAC4
:10774000900E287402F0900D77E06003B401E922F6
:10775000E4FFFE12015E600C0FEF70010E09E9708C
:10776000F20A80EF22900F2AE06404600BE5962075
:10777000E7FB75961175974822900B4FE0FD7F054A
:107780001274C6900B50E0FD7F0A0274C6AFFA7EF9
:1077900000ADF97C00ABFAEBB507F2EFFEEDFF228E
:1077A00075A5FF7590800000D2A000E4F59000C29E
:1077B000A022E4900B52F0A3F0C292D2931277A0D1
:1077C000D2A8227F05127340900B4F12733C900B8E
:1077D00050EFF022E4900C5BF0A3F0900B47F09098
:1077E0000B40F022E4FFFE0FBF00010EBE01F8BF08
:1077F000F4F522900CD9E004F07006900CD8E00467
:10780000F022900CD9E004F07006900CD8E004F05F
:1078100022D287D28375E40BD288D2A8D2AF2212AB
:107820007856127811E4F590C2A0D2A1227811E620
:1078300070FB781176018F9922E4900C5BF0A3F035
:107840000276617F0D7E001273017F00221275B3F4
:10785000E59130E7FB22C2A143A60743E240227F25
:10786000021271D1024ECC7F021271D10251DE7F21
:10787000011271D10258467F011271D10248117F65
:10788000011271D102438D7F011271D1023BEE7F53
:10789000011271D10262A47F011271D1023D49E44B
:1078A000FF1273727F0022AD077F1F0270C3E49046
:1078B0000F2BF022900E7AE0FF22E4900E7AF02255
:1078C0007F1C127340227F0C127340227F131273AD
:1078D00040227F0A026A8C7F09026A8C7F08026A52
:1078E0008C7F020278A77F9D0275FC7F9E0275FC4B
:1078F0007F800275FC75A59F227F012202791D02FF
:10790000535C02714B0265E7025F2B025FC20255B6
:10791000877F00227F00220232AD2222222222FF14
:1079200078FCFF78FCFF78FCFF78FCFF78FCFF78A0
:10793000FCFF78FCFF78FCFF78FCFF78FCFF78FC0C
:10794000FF78FCFF78FCFF78FCFF78FCFF78FCFFF9
:1079500078FFFF78FCFF78FCFF78FCFF78FCFF786D
:10796000FCFF78FCFF78FCFF7902FF78FCFF7905CB
:10797000FF78FCFF7908FF78FCFF78FCFF78FCFFBC
:1079800078FCFF78FCFF78FCFF78FCFF78FCFF7840
:10799000FCFF78FCFF78FCFF78FCFF78FCFF78FCAC
:1079A000FF78FCFF78FCFF78FCFF78FCFF78FCFF99
:1079B00078FCFF7720FF78FCFF786FFF78FCFF787A
:1079C00077FF78FCFF787FFF78FCFF78FCFF78FC7E
:1079D000FF7887FF78FCFF788FFF78FCFF4252FF2B
:1079E00078FCFF064DFF78FCFF7738FF78FCFF78C6
:1079F00097FF78FCFF7867FF78FCFF785FFF78FCE3
:107A0000FF78FCFF78FCFF78FCFF78FCFF78FCFF38
:107A100078FCFF78FCFF78FCFF78FCFF78FCFF72B5
:107A2000C6FF78FCFF790BFF78FCFF790EFF78FC2E
:107A3000FF78FCFF78FCFF78FCFF78FCFF78FCFF08
:107A400078FCFF78FCFF78FCFF78FCFF78FCFF787F
:107A5000FCFF78FCFF78FCFF78FCFF78FCFF78FCEB
:107A6000FF78FCFF78FCFF78FCFF78FCFF78FCFFD8
:107A700078FCFF78FCFF78FCFF78FCFF78FCFF784F
:107A8000FCFF78FCFF78FCFF78FCFF78FCFF78FCBB
:107A9000FF78FCFF78FCFF78FCFF78FCFF78FCFFA8
:107AA00078FCFF78FCFF78FCFF78FCFF78FCFF781F
:107AB000FCFF78FCFF78FCFF78FCFF78FCFF78FC8B
:107AC000FF78FCFF78FCFF78FCFF78FCFF78FCFF78
:107AD00078FCFF78FCFF78FCFF78FCFF78FCFF78EF
:107AE000FCFF78FCFF78FCFF78FCFF78FCFF78FC5B
:107AF000FF78FCFF78FCFF78FCFF78FCFF78FCFF48
:107B000078FCFF78FCFF78FCFF78FCFF78FCFF78BE
:107B1000FCFF78FCFF78FCFF78FCFF78FCFF78FC2A
:107B2000FF78FCFF78FCFF78FCFF78FCFF78FCFF17
:107B300078FCFF78FCFF78FCFF78FCFF78FCFF788E
:107B4000FCFF78FCFF78FCFF78FCFF78FCFF78FCFA
:107B5000FF78FCFF78FCFF78FCFF78FCFF78FCFFE7
:107B600078FCFF78FCFF78FCFF78FCFF78FCFF785E
:107B7000FCFF78FCFF78FCFF78FCFF78FCFF78FCCA
:107B8000FF78FCFF78FCFF78FCFF78FCFF78FCFFB7
:107B900078FCFF78FCFF78FCFF78FCFF78FCFF782E
:107BA000FCFF78FCFF78FCFF78FCFF78FCFF78FC9A
:107BB000FF78FCFF78FCFF78FCFF78FCFF78FCFF87
:107BC00078FCFF78FCFF78FCFF78FCFF78FCFF78FE
:107BD000FCFF78FCFF78FCFF78FCFF78FCFF78FC6A
:107BE000FF78FCFF78FCFF78FCFF78FCFF78FCFF57
:107BF00078FCFF78FCFF78FCFF78FCFF78FCFF78CE
:107C0000FCFF78FCFF78FCFF78FCFF78FCFF78FC39
:107C1000FF78FCFF78FCFF78FCFF78FCFF78FC1213
:107C200001100100000040251329C00000010200DE
:107C3000010902290001010080AF090400000203CC
:107C40000000000921010100012242020705810311
:107C500040000A0705020340000A0600FF0901A1CF
:107C60000185109502750826FF0015000901910293
:107C700085119530750826FF0015000901810285E0
:107C8000319502750826FF00150009019102853221
:107C9000953F750826FF001500090181028533957F
:107CA0003F750826FF0015000901910285349502F1
:107CB000750826FF001500090181028518950275D7
:107CC0000826FF0015000901910285199502750823
:107CD00026FF001500090181028535953F750826AC
:107CE000FF0015000901910285369503750826FFEE
:107CF0000015000901810285379507750826FF00E8
:107D00001500090191028538953F750826FF001579
:107D10000009018102851C9502750826FF001500E7
:107D200009019102851D9505750826FF00150009BA
:107D3000018102851A9505750826FF0015000901C5
:107D40009102851B9502750826FF00150009018127
:107D500002853F950C750826FF0015000901910268
:107D60008540950C750826FF0015000901810285E4
:107D700047953F750826FF001500090191028548C7
:107D80009502750826FF00150009018102854995B5
:107D90000C750826FF001500090191028550953FDA
:107DA000750826FF001500090181028541953F7580
:107DB0000826FF001500090191028542953F7508CC
:107DC00026FF0015000901810285439502750826EA
:107DD000FF001500090191028544953F750826FFB3
:107DE00000150009018102853B9507750826FF00F3
:107DF000150009019102853E9502750826FF0015C0
:107E00000009018102853D9506750826FF001500D1
:107E100009019102853C9502750826FF00150009AD
:107E200001810285459509750826FF0015000901A5
:107E3000910285469504750826FF00150009018109
:107E4000028555953F750826FF001500090191022E
:107E500085569502750826FF0015000901810285E7
:107E600058953F750826FF001500090181028557C6
:107E70009501750826FF00150009019102855A95A4
:107E80003F750826FF001500090181028559953FBD
:107E9000750826FF00150009019102C005030904B9
:107EA000000A0341004D005300200000000E034172
:107EB0000053003300390039003100000000001089
:107EC0002120423063408450A560C670E78108914C
:107ED00029A14AB16BC18CD1ADE1CEF1EF123102D3
:107EE000103273225252B5429472F762D69339839C
:107EF00018B37BA35AD3BDC39CF3FFE3DE246234E3
:107F0000430420140164E674C744A45485A56AB5EB
:107F10004B85289509E5EEF5CFC5ACD58D365326B2
:107F2000721611063076D766F6569546B4B75BA73B
:107F30007A97198738F7DFE7FED79DC7BC48C45842
:107F4000E5688678A70840186128023823C9CCD98B
:107F5000EDE98EF9AF89489969A90AB92B5AF54A12
:107F6000D47AB76A961A710A503A332A12DBFDCBDB
:107F7000DCFBBFEB9E9B798B58BB3BAB1A6CA67CA2
:107F8000874CE45CC52C223C030C601C41EDAEFD2B
:107F90008FCDECDDCDAD2ABD0B8D689D497E976EF2
:107FA000B65ED54EF43E132E321E510E70FF9FEF7B
:107FB000BEDFDDCFFCBF1BAF3A9F598F7891888120
:107FC000A9B1CAA1EBD10CC12DF14EE16F10800017
:107FD000A130C220E3500440257046606783B99306
:107FE00098A3FBB3DAC33DD31CE37FF35E02B11267
:107FF0009022F332D24235521462777256B5EAA516
:10800000CB95A88589F56EE54FD52CC50D34E224B6
:10801000C314A004817466644754244405A7DBB7E5
:10802000FA879997B8E75FF77EC71DD73C26D33606
:10803000F2069116B06657767646155634D94CC975
:108040006DF90EE92F99C889E9B98AA9AB58444856
:10805000657806682718C008E1388228A3CB7DDB45
:108060005CEB3FFB1E8BF99BD8ABBBBB9A4A755AA6
:10807000546A377A160AF11AD02AB33A92FD2EEDD5
:108080000FDD6CCD4DBDAAAD8B9DE88DC97C266CF6
:10809000075C644C453CA22C831CE00CC1EF1FFF25
:1080A0003ECF5DDF7CAF9BBFBA8FD99FF86E177E46
:1080B000364E555E742E933EB20ED11EF001000076
:0180C00000BF
:00000001FF
